:020000040001F9
:1090000070390020C1930100C9930100CB93010086
:10901000CD930100CF930100D19301000000000027
:10902000000000000000000000000000D3930100D9
:10903000D593010000000000D7930100D9930100EF
:1090400041970100DB930100B19A0100DB9301001D
:10905000DB9301000000000079950100DB93010023
:10906000DB930100DB930100DB930100DB93010044
:10907000DB930100DB930100DB930100DB93010034
:10908000DB93010099970100DB930100DB93010062
:10909000BD970100DB930100C1970100DB93010044
:1090A000DB930100DB9301000000000000000000E2
:1090B000DB930100DB9301000000000000000000D2
:1090C00000000000000000000000000000000000A0
:1090D0000000000000000000000000000000000090
:1090E0000000000000000000000000000000000080
:1090F0000000000000000000000000000000000070
:10910000000000000000000000000000000000005F
:10911000000000000000000000000000000000004F
:10912000000000000000000000000000000000003F
:10913000000000000000000000000000000000002F
:10914000000000000000000000000000000000001F
:10915000000000000000000000000000000000000F
:1091600000000000000000000000000000000000FF
:1091700000000000000000000000000000000000EF
:1091800000000000000000000000000000000000DF
:1091900000000000000000000000000000000000CF
:1091A00000000000000000000000000000000000BF
:1091B00000000000000000000000000000000000AF
:1091C000000000000000000000000000000000009F
:1091D000000000000000000000000000000000008F
:1091E000000000000000000000000000000000007F
:1091F000000000000000000000000000000000006F
:10920000DFF80CD000F07AF90048004731D80100AF
:109210007039002030B450E8012F93B2C489234440
:109220008489A34228BF1B1B0489A34202BFBFF34A
:109230002F8F002007E0C3EA020340E80134002C2E
:10924000E9D14FF001000A6030BC704750E8012FAF
:10925000C2EA024240E801210029F7D1704730B448
:1092600050E8022F1FFAA2F3C488A34202BFBFF343
:109270002F8F00200DE0C48923448489A34228BF96
:109280001B1BC2EA034340E80234002CE8D14FF034
:1092900001000A6030BC704750E8022FC2EA224247
:1092A00040E802210029F7D17047034653E8022F16
:1092B000D988B2EB324F4FF0000017BF92B241EAAB
:1092C000014142EA014104E05A68B2EB324F08BF63
:1092D000012043E80212002AE8D1704730B4044666
:1092E00054E8000F0D4644E80053002BF8D11560F8
:1092F00030BC704730B4044654E8000F40EA010522
:1093000044E80053002BF7D1156030BC704730B4EF
:10931000044654E8000F00EA010544E80053002B1E
:10932000F7D1156030BC704730B4044654E8000FE4
:1093300080EA010544E80053002BF7D1156030BCEA
:10934000704730B4044654E8000F00EB010544E8D0
:109350000053002BF7D1156030BC704730B4044681
:1093600054E8000FA0EB010544E80053002BF7D1AF
:10937000156030BC704770B404464FF0000054E8EC
:10938000006F0D68AE4207BF44E80023012044E8A7
:1093900000630E60002B1CBF0020F0E770BC70471C
:1093A00030B4044654E8000F88422CBF451A0546E5
:1093B00044E80053002BF5D1156030BC7047000025
:1093C0000648804706480047FEE7FEE7FEE7FEE75F
:1093D000FEE7FEE7FEE7FEE7FEE7FEE7C5970100D2
:1093E000019201002DE9F05F0546002092469B4660
:1093F00088460646814640241BE0284641464746AB
:10940000224600F06BF853465A46C01A914110D3D9
:1094100011461846224600F016F82D1A67EB01088F
:109420004F4622460120002100F00DF817EB0009FD
:109430004E41201EA4F10104DFDC484631462A4695
:109440004346BDE8F09F202A04DB203A00FA02F1EF
:10945000002070479140C2F1200320FA03F3194322
:1094600090407047004870477831020040EA01039D
:109470009B0703D009E008C9121F08C0042AFAD2CA
:1094800003E011F8013B00F8013B521EF9D270478E
:10949000D2B201E000F8012B491EFBD27047002236
:1094A000F6E710B513460A4604461946FFF7F0FFE3
:1094B000204610BD421C10F8011B0029FBD1801A68
:1094C000704730B504460020034600E05B1C934221
:1094D00003D2E05CCD5C401BF8D030BD202A04DB19
:1094E000203A21FA02F00021704721FA02F3D0401D
:1094F000C2F120029140084319467047064C074DBF
:1095000006E0E06840F0010394E807009847103453
:10951000AC42F6D3FFF778FE203902004039020052
:1095200070B58C1810F8015B15F0070301D110F825
:10953000013B2A1106D110F8012B03E010F8016B52
:1095400001F8016B5B1EF9D12B0705D40023521ED5
:109550000DD401F8013BFAE710F8013BCB1A921C3D
:1095600003E013F8015B01F8015B521EF9D5A1423B
:10957000D8D3002070BD00002DE9F04700268AB046
:10958000DFF85091B0464FF48075012437460696B7
:10959000284605F0F1F938B1D9F80403204203D088
:1095A000284605F0DFF926432D1D64007F1CADB26F
:1095B000082FEDD34FF4BE74204605F0DDF948B115
:1095C000204605F0CFF946F0004606AA012100200A
:1095D00005F0B4F9404D16F0FF0F15D00127002417
:1095E00037420DD009EB8401D1F81005D1F81015E0
:1095F000C0F3042055F82420C1F3014102B1904783
:109600007F00641C082CEBD3002E5FDA4FF0FF3094
:10961000CDF8108054E0281910F8507F90F9000020
:1096200027F0C008401C3BD007A9404604F043FC8B
:1096300010B34FEA9719404602F052F855F82070DF
:109640001FB1B9F1030F03D006E0B9F1030F27D121
:1096500004A9404604F037FC4FF0A04101EB88001C
:10966000D0F8000706A9C0F3014A404604F023FCE5
:1096700018B1BAF1020F03D012E0BAF1030F0FD103
:10968000B9F1030F08D1BAF1020F1DD002214046F3
:1096900005F038F9761CF6B217B149464046B8478E
:1096A000641C042CB7D3002E10D06A460121002080
:1096B00005F044F906990098884207D0069004986E
:1096C000002634460790A6E70321E0E70AB0BDE88C
:1096D000F0870000006000400829002000F01F0211
:1096E000012191404009800000F1E020C0F8801283
:1096F000704700F01F02012191404009800000F1F5
:10970000E020C0F80011704700F01F0201219140D5
:109710004009800000F1E020C0F8001270474907BE
:10972000090E002806DA00F00F0000F1E02080F8B2
:10973000141D704700F1E02080F80014704700000D
:1097400070B54FF48076304604F0C6FC114CB50578
:1097500060B1304604F0C7FC0120C5F80803607909
:1097600020B9012060712168002088474FF482767B
:10977000304604F0B1FC00280AD0304604F0B3FCB7
:109780000220C5F808032168BDE8704001200847A1
:1097900070BD0000041F002007480021C0F84011E0
:1097A000C0F84411C0F84811C0F84C11C0F80011BD
:1097B000C0F8041108F0F2BD0010014008F03CBDF3
:1097C00005F02EBEF0B5A848A74B012600781B1D5A
:1097D0001A1D4FF0805106280BD11C78240708D1A0
:1097E0001478C4F30314032C06D0042C04D0052CE5
:1097F00002D0062807D011E0B1F824439B4DC4F3F2
:1098000004242C6002E01C78240707D11478C4F3E8
:109810000314032C02D1974D954C6C67D1F830514D
:10982000D1F84442944FC4F342343C6006280CD132
:109830001C78240709D11478C4F30314032C04D131
:109840008E4C276827F0807727604FF080470024F0
:10985000C7F80C41C7F81041874F3F1F3C600628EE
:1098600007D11F783F0704D11778C7F30317032FD9
:1098700002D0062808D01FE0DFF8FCC103270CF156
:10988000640CCCF8007007E01F783F0714D11778FC
:10989000C7F30317032F0FD1DFF8E4C10527CCF876
:1098A0000070774F78373E60754F08373C600CF199
:1098B000040C3F27CCF80070724F3F68DFF8C8C136
:1098C000CCF800706F4F3F1D3F680CF1040CCCF8D2
:1098D00000706C4F08373F680CF1040CCCF8007036
:1098E000684F0C373F680CF1040CCCF80070654FE2
:1098F00010373F680CF1040CCCF80070614F14373E
:109900003F680CF1040CCCF800705E4F18373F68CC
:10991000DFF874C10CF1200CCCF80070594F1C37E3
:109920003F680CF1040CCCF80070564F20373F68AC
:109930000CF1040CCCF80070524F24373F680CF146
:10994000040CCCF800704F4F28373F680CF1040C22
:10995000CCF800704B4F2C373F680CF1040CCCF85E
:109960000070484F30373F68DFF81CC10CF1400CE5
:10997000CCF80070434F34373F680CF1040CCCF83E
:109980000070404F38373F680CF1040CCCF8007081
:109990003C4F3C373F680CF1040CCCF80070394F59
:1099A00040373F680CF1040CCCF80070DFF8DCC0E5
:1099B000FB27CCF80070062813D11F783F0710D181
:1099C0001778C7F30317032F03D0042F01D0052FF7
:1099D00007D1D1F85872DFF8B8C007F04F07CCF8BC
:1099E00000702C480268D20702D06FF001020260BA
:1099F000062D08D1D1F83401062804D12648016883
:109A000041F4806101604FF01021D1F8000200287C
:109A100003DBD1F80402002822DA204A166020482D
:109A20000368002BFCD01523C1F800320568002D17
:109A3000FCD0C1F8043201680029FCD01460016830
:109A40000029FCD0BFF34F8F0C48F0380168154A4D
:109A500001F4E06111430160BFF34F8F00BFFDE7E8
:109A6000124911480860F0BDE00F00F04035014098
:109A70000DF0ADBA00C007403C050040FCED00E031
:109A8000105600400404001020C5004018F50040A6
:109A9000E40E0040000400403C17004004E5014093
:109AA00000E401400400FA050090D0032C200020BF
:109AB0000149024808F0FCBC642900200020004055
:109AC00002E008C8121F08C1002AFAD17047704787
:109AD000002001E001C1121F002AFBD170470000E5
:109AE0000121202803DA81400548014003E0402895
:109AF00002DA2038814009B1012070470020704708
:109B0000FC06FFBD082806D228B1012803D004288E
:109B100001D0012070470020704710B560B159B1E5
:109B200002780B785208B2EB530F05D10622401C85
:109B3000491CFFF7C6FC08B1002010BD012010BD74
:109B4000800701D00020704701207047C3688B4216
:109B500006D811440069491E814201D8012070478E
:109B60000020704710B501220221002001F0C8FB3F
:109B700008B1072810D107220221012001F0C0FB03
:109B800008B1072808D100210A22084601F0B8FBD5
:109B900008B1072800D1002010BD000000B5ABB00F
:109BA000AC216846FFF77BFC02208DF80000012005
:109BB0008DF8020005218DF803101249ADF8180048
:109BC00007918DF879008DF87C008DF87D004FF4B9
:109BD00048602490282144F250602291259040F65C
:109BE000B8310948239129906946084800F028FCBB
:109BF00008B100F027F90121044800F01EFC2BB049
:109C000000BD00004C1B0020C1F901008421002090
:109C10002DE9F04750B125480321008801EB0040B1
:109C200023A105F08FF807F0AFFA37E04FF6FF7881
:109C3000424610212248FFF72BFC224D0820044603
:109C4000A8601F4F05F10806404607F047F90021BC
:109C5000B1463160464608E0D9F800104B00491C77
:109C6000C9F80010F85207F039F9B04201D0641E6B
:109C7000F2D21348A96807F0F7FA08B100F0E2F849
:109C80000F48A96806F0F2FF062802D008B100F0DC
:109C9000D9F80B480321B83800F0B9FC002803D0EC
:109CA000BDE8F04700F0CEB8BDE8F087782000208E
:109CB000457261736520626F6E647321000000005D
:109CC0003C220020481B002070B58CB015460E4683
:109CD00000236C46C3F10F01415CE1545B1C102B67
:109CE000F8D30D2104F11000FFF7D9FB0020C0F1DB
:109CF0000F02315C2244401C11740328F7D36846DC
:109D000046DF0020C0F10F01214491F820102954B2
:109D1000401C0328F6D30CB070BD022001F0D0B96E
:109D20000149097900F01EBED81E002070B500243C
:109D3000064D06E06868012110F8340005F04AFC81
:109D4000641C28788442F5D3002070BD101F0020C9
:109D5000F8B515460C460646052A01D20720F8BD7F
:109D600005F034FD18B905F0F9FC0028F7D11249C7
:109D700000224E600C708D60C1E90422C1E9062208
:109D80000E4D0DE006EBC4002968009181788DF836
:109D9000011000780A4A694605F06EFC0028DED101
:109DA000641EE4B2EED2BDE8F84004480021054A42
:109DB000001D00F0D9B80000101F0020FC2D02008B
:109DC000B9CA0100ADBE010072B605F071F800BF5E
:109DD00004F0A8FE0028FBD1104C0121208801EBE3
:109DE00000400FA104F0AEFF10480068C00700D08B
:109DF00000BE2088022101EB00400DA104F0A2FF6B
:109E0000BFF34F8F0948E43801680D4A01F4E0615F
:109E100011430160BFF34F8F00BFFDE778200020A2
:109E2000466174616C206572726F7200F0ED00E043
:109E300053797374656D207265736574000000005A
:109E40000400FA050EB500210091CDE901106A4623
:109E500044F20100FFF7B8FF0EBD00002DE9F84FF6
:109E6000254C8146924660880E46814241D80027A3
:109E70004FF6FF788DF80070684600F005F92278FB
:109E80006078A188884201DA401C00E00020C0B25E
:109E9000904204D19DF8000000F01AF927E065789F
:109EA0006078884201DA401C00E0002060709DF874
:109EB000000000F00DF9454519D0A068B9F1000F78
:109EC00040F835A00DD066B16188E068324605FBE8
:109ED00001004946FFF7CAFAA06800EBC50086807A
:109EE00002E000EBC50087800020BDE8F88F042069
:109EF000FBE70920F9E70000301F002010B50E4CE9
:109F000003E0401C00E0002020702078617881424E
:109F100010D022786188E068A36802FB010003EB9F
:109F2000C20153F83220898890472078A18888425E
:109F3000E9DAE6E710BD0000301F002030B5CB00A5
:109F400008339DB293074FF0000401D0072030BDC5
:109F5000044B9A602A44DA605C701C7058809980C7
:109F6000002030BD301F0020074B9B7823B12AB161
:109F700020B10068037C1BB10820704707207047A0
:109F80004174426100207047A829002070B507F095
:109F90001DFC104800240B21047044700E4D81708C
:109FA00014206C602C706C70FFF798FB0721142054
:109FB000FFF7B5FB1420FFF79CFB0848046007215E
:109FC0001120FFF7ACFB0548001F0068A8600020C7
:109FD00070BD0000A8290020401F00200815014086
:109FE0002DE9FC47DFF8789099F8023073B368B335
:109FF000052902D20720BDE8FC87436933B3437CBF
:10A00000012B25D0002704460025884616468DF8EA
:10A010000050684600F038F801A808F095FBC8B178
:10A02000012101700F4944600968C0E90218C0E9C4
:10A0300004769DF8040089F801009DF8000000F006
:10A0400047F81420FFF760FB2846D4E70820D2E742
:10A050000F46D8E704259DF8000000F039F8F3E733
:10A06000A8290020041501400649897839B130B18A
:10A07000416921B100210174022108F06BB9082067
:10A0800070470000A829002030B5EFF3108172B6A8
:10A090000D4A9468012324B10370002900D162B6EF
:10A0A00030BD93604FF0E023D3F88051074C25403A
:10A0B0001560C3F88041D3F8844154605A17C3F83F
:10A0C000842100220270E8E7B42A0020FC06FFBDCC
:10A0D0000B498A68002A11D000280FD1EFF31080B5
:10A0E00072B60B684FF0E022C2F800314B68C2F83C
:10A0F000043100228A60002800D162B67047000057
:10A10000B42A00202DE9F041064608680C46411C9F
:10A110004FF0A0474FF0010506D005FA00F1C7F84F
:10A120000815206804F0E4FB6068411C02D000219F
:10A1300004F0D5FB3168A069C1F82405607D217D5C
:10A1400032680843C2F86C05D4E900123068C0F8E0
:10A150000C15C0F81425207D012815D1A068411CDC
:10A1600002D0002104F0BBFBE068411C05D0854013
:10A17000C7F80855E06804F0BBFBD4E90212306868
:10A18000C0F80825C0F81015BDE8F08103F0ACBA9E
:10A190002DE9F047074600888EB0804602F020FF88
:10A1A000824604462D4800252A460178404600F0A4
:10A1B000F1FB7879400734D501254FF6FF7603ABE4
:10A1C0002A460721504606F0F7F8010004D0404621
:10A1D00007F0FCFC00252BE0B1463146049802F064
:10A1E00052FE064648450FD004460146404602F05E
:10A1F000E1FE4046FFF794FD30B9404607F0B8FC59
:10A200004046FFF78DFD48B122460721504606F033
:10A2100049F9010003D0404607F0D8FC00254E451F
:10A2200006D0404606F0ACFA10B1504602F0C4FE2B
:10A2300002208DF81800ADF81A807879400701D512
:10A24000012000E002208DF820008DF8215006A8A2
:10A2500002F034F80EB0BDE8F0870000D81E0020F0
:10A260002DE9FC47002517880646158090F82D003B
:10A270001446894630B13A462146484600F0F6FC7D
:10A28000051E09D1B0784FF00C0A18B32088C846D3
:10A29000001DB84202D95046BDE8FC87684679DF08
:10A2A0000028F9D12088032108F8001020881921FE
:10A2B000401C80B2208008F800102088401C80B22A
:10A2C000208000EB0801BDF8000008F06BF9218840
:10A2D00008442080F0780222C8B1218896F9033022
:10A2E00001F1030C4846BC45D5D8425421884FF0B3
:10A2F000010C491C89B2218000F801C02188491C49
:10A3000089B2218009F801302088401C20807068C3
:10A31000B8B1218890F9003001F1030C4846BC45E2
:10A32000B9D8425421880A22491C89B2218042545A
:10A330002188491C89B2218009F801302088401CFD
:10A340002080308950B1CDE900474B4606220221DA
:10A3500006F1080008F010FA051E9DD1308A50B1B0
:10A36000CDE900474B460722032106F1100008F013
:10A3700003FA051E90D1308B50B1CDE900474B4612
:10A380001522142106F1180008F0F6F9051E83D1F4
:10A39000306A30B13B462246494601F07EFA051E3E
:10A3A000DBD1706A30B13B462246494603F03EFBA2
:10A3B000051ED2D196F82C0038B13B4622464946BC
:10A3C000304607F02DFC051EC7D1307838B13B462A
:10A3D00022464946304603F0AFFB051EBDD1284654
:10A3E0005AE718B504460020ADF8000013466A4647
:10A3F000204600F006F8002802D0BDF800002044F6
:10A4000018BD70B588B182B10024158803E0065DDF
:10A41000641C3444A4B2A54203D8061976789E423F
:10A4200001D08C42F3D38C4201D3002070BDA11C1B
:10A430001180005D401E80B270BD80F83010704702
:10A440002DE9F0410D00044606D02CB195F87A00B4
:10A450000026012803D006E00E20BDE8F08195F823
:10A460009800012829D0D5F8A000042825D0D5F8D7
:10A470009C00042821D04FF00108A6702C2205F181
:10A480007801201DFEF7F2FF84F83060D5F8A400B3
:10A490006063D5F8A800A0634FF6FF70A4F8A80089
:10A4A00004F19400C4F8A400C4F8AA60A4F8AE6053
:10A4B00084F8B060207810B104E00720CDE7FF20D9
:10A4C00084F8540004F155011F27C4F89410A4F82F
:10A4D000987004F198022846FFF7C2FE0028BCD10C
:10A4E00015F13C0F0ED004F17401C4F89C10A4F8CF
:10A4F000A07004F1A00205F13C00FFF7B1FE0028B6
:10A50000ABD103E0C4F89C60A4F8A06084F851804B
:10A51000208BA4F8480084F83C80266484F85060BE
:10A5200060696064454604F13C02002104F1540076
:10A5300072DF002891D125708FE710B50288102AAC
:10A540001BD0112A20D0262A1DD1007A0C460128C2
:10A5500001D0022817D1A0780521401CB0FBF1F2F0
:10A5600001FB1201204600F052F800280BD0A16B2D
:10A57000002908D0BDE810400847C27B012A02D15B
:10A580008088A1F8A80010BD0C46002184F8B21004
:10A590008088B4F8A8108842F5D120790028F2D13B
:10A5A0000121DFE710B50C46022801D0032810D1A5
:10A5B000607800280DD000206070A178204600F05F
:10A5C00026F8002805D0A16B002902D0BDE8104074
:10A5D000084710BD10B5044690F8540074DF012000
:10A5E00084F8B200002084F8B40084F850000621FA
:10A5F000204602F069F8002808D1A178204600F032
:10A6000006F810B1A16B01B18847002010BD2DE9FB
:10A61000F05F044600780F4638B1A770002003F0C1
:10A620009FFF012620B16670F4E00820BDE8F09F8E
:10A630000025C4F8AA50A4F8AE5084F8B050A07910
:10A6400010B1A078012806D0E07968B1A07801287F
:10A6500001D0022808D1616B21B184F8B1600820D3
:10A66000884701E084F8B15004F1AB0100200A5C96
:10A670000AB1304603E0401C0628F8D300204FF012
:10A6800002084FF0030A4FF0040B012F06D0022FEF
:10A690000CD0032F0FD0042F15D110E0A17929B1D0
:10A6A00094F8241011B908B130460DE0E17911B1E8
:10A6B00008B1404608E0207A08B1504604E0607ACC
:10A6C00008B1584600E02846A070616B41B10328EC
:10A6D00001D0042804D1607910B194F8B200A0B17F
:10A6E00084F8B35004F13C0018210746FEF7D7FE6A
:10A6F00004F12C0084F83C60814606F0CDF958B195
:10A7000094F82C0084F8510008E084F8B45084F8E0
:10A71000B36007208847E5E784F8516094F8240087
:10A7200050B1484606F0B8F920B194F8280084F8F2
:10A73000520001E084F8526084F85050A27804F18D
:10A74000AA0104F19409052A4DD2DFE802F065035D
:10A750000F1B320084F83160C4F8A450C4E910150E
:10A7600084F83C808020A4F848003EE084F83180E2
:10A7700087F800A0228ABA81C4F8A4507960E16801
:10A78000B96032E06069B860208BB8813D4684F8DA
:10A790003C60204607F0B4FF40B185F814800421E6
:10A7A000204601F091FFF0B9052115E084F831A0B1
:10A7B00017E0E069B860208CB8813D4684F83C60C1
:10A7C000204607F09DFF50B185F8148004212046F3
:10A7D00001F07AFF38B9062184F8311001E084F8DD
:10A7E00031B0C4F8A490A07878B13A4604F154008E
:10A7F000D4F8A41072DF00287FF418AF94F830105A
:10A8000094F8540073DF0028F6D1616B11B194F80D
:10A8100031008847002009E784F83150F5E790F8C7
:10A82000B330009933B1002380F8B3300A4303D02A
:10A83000012102E008207047002180F8B4100020B8
:10A840007047000070B5040012D001461C22144865
:10A85000FEF70CFE1248134D0560206850B17ADFF8
:10A86000002806D12068016829604068686005E01A
:10A870000E2070BD0B487BDF0028FAD108484FF648
:10A88000FF711438084A20F8041B05493439016067
:10A890000021FFF769FB0028EBD0032070BD00000A
:10A8A000EC2200208C1E00209926020010B50446E0
:10A8B00000F090F8002805D02146BDE8104002487D
:10A8C00003F05DBA10BD00001823002070B51546D6
:10A8D0000E46044607F020FF002809D0054800EB8B
:10A8E000840080692A463146BDE8704001F02ABFE5
:10A8F00070BD00000823002010B5044600F06AF87F
:10A90000002805D02146BDE81040024803F037BAC0
:10A9100010BD00001C23002010B5002400F05AF8E0
:10A9200000B10124204610BD70B50546002400F09A
:10A9300051F838B12946044803F021FA08B102243D
:10A9400000E00124204670BD1023002010B518211E
:10A95000034803F0EFF9182800D0C0B210BD000082
:10A960000823002070B505460C46084607F0D4FEC3
:10A9700060B1284600F02EF840B10548294600EBAA
:10A980008400BDE87040183003F0F9B9002070BDB4
:10A990000823002070B5054614460E46084607F009
:10A9A000BBFE002812D0284600F014F800280DD075
:10A9B0000748294600EB860018301CB1BDE87040FE
:10A9C00003F0E8B9BDE8704003F099B970BD00002C
:10A9D00008230020142801D30020704701460148B5
:10A9E00003F0CDB90C23002010B5044600F032F876
:10A9F00020B12189A0890022A1DF10BD052010BD52
:10AA000038B181811AB151884181118801810020BA
:10AA100070470E2070470000B8B1B1B14A68A2B1CA
:10AA20000A6892B10A4A0123937041F60503138024
:10AA30000A680260496841604FF6FF718181002118
:10AA400001814181024800F087B80E207047000064
:10AA5000F61E00200089002800D00120704710B5A4
:10AA60000A46014610460A8886B0112A06D0362AC0
:10AA70001BD106B0BDE8104001F00CB90446808936
:10AA80008988884202D14FF6FF70A0812046FFF7E7
:10AA9000E1FF002809D002208DF8000022686946F5
:10AAA0002046904700202081608106B010BD000044
:10AAB00070B586B0044601208DF800004888ADF8D6
:10AAC0000200087801F10E0340BB8888A0F5C0524F
:10AAD000053A23D18879012820D142F62B25087A1E
:10AAE0000FE000BF02EBC20601EB4606F689AE425C
:10AAF00006D11889ADF804005889ADF8060002E0C7
:10AB0000521C9042EED808480321008801EB004017
:10AB100006A104F017F900208DF8000022686946AC
:10AB20002046904706B070BD4C20002043757272DD
:10AB3000656E742054696D6520536572766963652E
:10AB400020646973636F7665726564206174207038
:10AB50006565722E0000000070B540B10C4D29787B
:10AB600039B1044606F00CFE28B1002070BD0E205D
:10AB700070BD082070BDE868062807D20549226824
:10AB800001EB8001401C0A60E860EEE7042070BD24
:10AB9000941E00208023002040B10549002201239B
:10ABA000CA600B70C1E90102104670470E20704761
:10ABB000941E002070B504002DD000292BD0204811
:10ABC0000078002827D020880D46112815D030287D
:10ABD00004D0322807D033281ED109E0211D284691
:10ABE00005F0AEF918E0211D284604F077FF13E0C8
:10ABF000211D284605F0D8F80EE0A088B5F8CA1245
:10AC0000884209D1002085F8C70285F8C8024FF6AE
:10AC1000FF70A5F8CA0270BD95F8C8020028FAD0E6
:10AC200020883028F7D34F28F5D8A088B5F8CA1265
:10AC30008842F0D12846BDE8704001F0E9B9000033
:10AC4000941E002048B1084A137843B1D26832B14B
:10AC500090F8C7222AB1112070470E2070470820B3
:10AC6000704701F0D5B90000941E00207CB5054660
:10AC700008880C460930904201D90C207CBD6846FA
:10AC80006DDF0028FAD121880820685420881B2114
:10AC9000401C80B2208029542088401C80B2208033
:10ACA0002844DDF801100160BDF80510818020887E
:10ACB000801D80B220809DF80010490800D001213D
:10ACC00029542088401C208000207CBD38B5028893
:10ACD0000446212A3FD017DC26484FF00301264DB9
:10ACE0000088102A01EB004016D0112A0BD123A1B5
:10ACF00004F028F84FF6FF7024492880A2888B8939
:10AD00009A4200D1888138BD3B2A2ED0562AFAD1EA
:10AD10008088132176DF18E01DA104F013F80720C6
:10AD200000F010FB08B1FFF78DF81848A1882980C2
:10AD3000203003F059F908B1FFF784F817480022D2
:10AD40004FF400310068FFF74BF90028DBD0BDE875
:10AD50003840FFF777B800200090A08869468FDF61
:10AD60000028D0D0FFF76EF838BD8088132176DF39
:10AD7000EBE7000078200020481B00204469736343
:10AD80006F6E6E65637465642E00000058210020AC
:10AD9000436F6E6E65637465642E0000742C020050
:10ADA00010B51A4C0188606810290ED011292BD1DA
:10ADB000401E606028D1FEF7D5FE002824D021680F
:10ADC000002921D0BDE810400847D0B90021012258
:10ADD000084600F095FA08B107280FD10722022192
:10ADE000012000F08DFA08B1072807D104220221C2
:10ADF000002000F085FA20B1072802D0216801B1B7
:10AE000088476068401C606010BD0000841E002000
:10AE10002DE9F04701883B4E40F2F3194FF6FF75DC
:10AE200010291BD011293ED0122954D0502946D1C7
:10AE3000C188F289841D914241D1618902293ED1A4
:10AE40008688304602F0CEF9050038D004F10C00B7
:10AE500000F0F2F8A8B3294630464EE0C17B87885F
:10AE6000044601292BD1A846284602F0BBF905006B
:10AE700017D02F8000202872234843464A46016895
:10AE8000C5F80A104068C5F80E0004F1100105F17C
:10AE90000A0002F073FA6872F08900280FD129467F
:10AEA0002AE0042013E0808802F09CF9040006D018
:10AEB0006068FFF7D9F808B106F06CFE2580BDE8A0
:10AEC000F087FFE76868FFF7CFF80028F7D0BDE804
:10AED000F04706F05FBE87880646384602F082F9E2
:10AEE0000400ECD02B464A4606F1080104F10A00A2
:10AEF00002F044FA607221463846BDE8F04700F09F
:10AF000013BD0000EC2200208C1E00202DE9F04F24
:10AF10000746858802883D48012197B08346102A5C
:10AF200009D0112A49D01A2A6CD1387AB1EB101FF6
:10AF300045D2012244E0354C083CA068C0430B9048
:10AF400061680BA802F03FFF0B990CA800F086FC8B
:10AF50002C220CA96846FEF789FA0026E946A0468D
:10AF600010E000BF09EB46005FF00004B0F804A059
:10AF700008EB84005146001D02F0C1FE641C1D2C2C
:10AF8000F6D3761C0098B042ECD8142D05D317B038
:10AF90000420BDE8F04FFEF755BF2946584602F0A1
:10AFA000F9FE294608F1040002F0F4FEF87B0128BE
:10AFB00028D016482946001D15E029461AE000222F
:10AFC0000221B1EB101F01D2012600E000260F493B
:10AFD000083901F11000041D294682B102F0DAFEA1
:10AFE00036B12946204617B0BDE8F04F02F0D2BE78
:10AFF0002946204617B0BDE8F04F02F080BE02F0AF
:10B000007EFEF5E717B0BDE8F08F000010230020AA
:10B0100010B504460748007800280AD0204601F001
:10B0200065FE204606F054FE2046BDE8104001F0C3
:10B0300095BC10BDC81E0020007800F001007047CC
:10B040000149085C704700007C2C02000649095C3D
:10B050004FF0A040D0F81005C84010F0010000D01B
:10B06000012080F0010070477C2C02002DE9FC419A
:10B070000646C0074FF000050ED0104F00240122F5
:10B08000385D009500231146019503F0E9FB641C2F
:10B09000042CF4D300F046F8B0070DD5074E002479
:10B0A000361D0022305D032300951146019503F003
:10B0B000D7FB641C042CF4D3BDE8FC81782C02007F
:10B0C00007490B5C4FF0A041D1F8042501209840BE
:10B0D00020EA0203C1F808351040C1F80C0570479A
:10B0E000782C02000249085C012103F01CBC00001E
:10B0F000782C02000249085C002103F014BC000017
:10B10000782C02000649095C4FF0A040D0F80405F5
:10B11000C84010F0010000D0012080F0010070470D
:10B12000782C020010B500242046FFF7DBFF641CDA
:10B13000042CF9D310BD10B500242046FFF7DAFF28
:10B14000641C042CF9D310BD10B50246064B4FF019
:10B15000FF3000215C5C944201D1084610BD491CBF
:10B160000429F7D310BD00007C2C020070B50C4EF2
:10B170000C004FF0000530600BD0012000F06AF8A1
:10B1800008B1022004E0002000F064F800B10B20B8
:10B190002070706810B9FEF7E5FC0546284670BDC2
:10B1A000841E002010B5002000F0FEF908B106282A
:10B1B00006D1012000F0F8F908B1062800D10020DE
:10B1C00010BD00002DE9F0470D468146FFF7BCFF9A
:10B1D0000446042836D2DFF874801B481C4EA8F1C0
:10B1E0000C0725B3012D0ED0022D2BD104EB44000A
:10B1F00030444578002D25D0B968002922D0284652
:10B20000BDE8F047084704EB4401755C0E447178D3
:10B2100049B10E4A4FF40041093A8068FEF7E0FE5A
:10B2200008B987F80390B17808F80410E2E780685D
:10B23000FEF71AFF04EB4401314418F804008D783E
:10B24000A842D7D0BDE8F087802C0200801E0020E5
:10B250008C220020042801D2FFF7F8BE002070479E
:10B2600010B504281ED019494FF6FF7207288989A6
:10B2700023D00A2812D00E2827D1914225D0134876
:10B28000FFF7B2FB052820D1114803210088BDE853
:10B29000104001EB00400FA103F054BDBDE8104089
:10B2A00006F002BD15481321008876DF0BE0002868
:10B2B0000BD0BDE81040FEF7C5BD914205D1034853
:10B2C0002C30FFF787F90828F1D110BD5821002054
:10B2D0007820002043757272656E742054696D6524
:10B2E0002053657276696365206973206E6F7420E0
:10B2F000646973636F76657265642E00481B002075
:10B3000070B50023042810D20D4D00EB4004012A33
:10B3100002D101290CD00022094E00EB400030443C
:10B3200061B1012906D0022906D00723184670BD55
:10B330000E30C2B22A55F9E74270F7E78270F5E79E
:10B340008C220020044A014600201279D20702D044
:10B35000084600F04DB87047741E002070B50646D0
:10B360001E480024C0E90161B00720D50025012254
:10B3700011462846FFF7C4FF6D1C0446042D02D277
:10B38000002CF4D013E094B940F266620421144812
:10B39000FEF7DEFC04000AD1FEF7C8FC040006D16B
:10B3A0000F48104A0021001FFEF7DEFD0446F0079B
:10B3B00012D00120FFF75AFE74B909480A4A002149
:10B3C0000C38FEF7D1FD040006D10548074A0121DB
:10B3D0000838FEF7C9FD0446204670BD741E0020E3
:10B3E0008C2C020075B601005DD401001B9D01008C
:10B3F0002DE9F05F6A4C054600266078B34618B127
:10B4000084F801B002F012F8664F4FF47A694FF4F5
:10B41000C87A4FF00108182D62D2DFE805F0AC0CB5
:10B420000C31404D62676B746B74BE7D7D7D7D7D9C
:10B43000ACAFB2B5BEBE0020FFF764FE00284FF0EF
:10B44000000008D0FFF74EFE022D02D14FF4E1605C
:10B4500008E0484606E0FFF74DFE022D01D1C82066
:10B4600000E05046410CC0034FF4FA72801841F1DD
:10B470000001257052000023FDF7B4FF01462AE0C9
:10B480000020FFF73FFE00284FF0000004D0FFF738
:10B4900029FE4FF44870E5E7FFF72CFEDFE70020B8
:10B4A000FFF730FE00284FF0000002D0FFF71AFE31
:10B4B000CFE7FFF71FFED4E70020FFF723FE0028A9
:10B4C0004FF0000002D0FFF70DFE01E0FFF712FE83
:10B4D000257041F69A1100223868FEF781FD064674
:10B4E00046E00020FFF7ECFD257008E0002051E069
:10B4F00025703DE084F801800120FFF7E1FD002286
:10B5000040F6CD41E8E784F801800120FFF7D8FD3F
:10B5100000224FF48041DFE77868FEF7A5FD06467C
:10B52000D5F1110000D02EB10220FFF7DBFD84F829
:10B5300002B01DE0012816D980B2C8214843C117C6
:10B54000C90341EA5041C0034FF4FA72801841F137
:10B55000000152000023FDF745FF014600227868F4
:10B56000FEF73EFD06460220FFF7C4FD84F8028088
:10B570003046BDE8F09F01F059FFB9E701F056FFF2
:10B58000B4E701F053FF04E001F050FF0020FFF7A3
:10B59000B1FD0120FFF7AEFDAAE7FFF7CCFDA7E75D
:10B5A000741E0020802C0200012107F04CB900001D
:10B5B0002DE9F8430546861C00208DF800009046D2
:10B5C0000F464FF001096846FEF75EFD1B4C2068F0
:10B5D0003860D4E90001401AA16804F21C47081A37
:10B5E0000EE00121384602F0E8FB02F0D3F80146F4
:10B5F000384602F0E2FBD4E90001401AA168081ABB
:10B60000401C8642EDD8B8F1000F03D0052065F349
:10B61000891002E0062065F39F50A268216811405E
:10B6200004EB8101C8602068304420609DF8000070
:10B63000FEF74EFD4846BDE8F88300004C2D002083
:10B6400030B482680468531C8360A154D0E90112AD
:10B650008A4202D330BC02F0B0BD30BC704700005B
:10B66000034803C8814201D1012070470020704780
:10B670004C2D002000780221FFF7A4BD05494FF0B2
:10B68000FF32082841F8202002D3084480F84820DF
:10B690007047000008290020F0B54FF0FF3512B1C7
:10B6A0000023082601E008230C260C4C05E000BF0F
:10B6B00054F823707F1C04D05B1CB342F8D3284697
:10B6C000F0BD26185DB286F8305044F82310002AE9
:10B6D000F5D1E11881F84800F1E7000008290020C1
:10B6E0000249084490F93000704700000829002002
:10B6F00008B5024690F8C6020B4600EB8001C1EB8C
:10B70000801002EB400092F8C52242B1521ED2B224
:10B7100002EBC20100EB4102518A491C00E0C188E2
:10B72000ADF800100089ADF80200694618469DDFAB
:10B7300008BD70B504464FF6FF750A462846AC4270
:10B7400008D14FF480742146104605F083FBA042D7
:10B7500009D070BDFF2CFCD82146104605F06DFBCA
:10B7600008B1204670BD284670BD000070B5084C79
:10B77000050009D010342168002907D0086820602E
:10B78000496828468847F6E70834F4E770BD0000AA
:10B79000F4280020054A012120B1012805D191702B
:10B7A000FFF7E4BF51700020FAE77047F42800204B
:10B7B0002DE9F05F26484168F1B3DFF898B00E68D4
:10B7C0008146DBF8004087688078E11B21F07F45E7
:10B7D000ED1CB0B9DFF880804FF48030C8F8440326
:10B7E000C8F804031120FDF779FF1120FDF781FF50
:10B7F0004FF0010AC8F800A02F2003F0E3FE89F8FB
:10B8000002A0B54200D23546124BE8193C3320F075
:10B810007F401860DBF800105A46091B21F07F4179
:10B82000001B20F07F40C91C81420FD910681860AE
:10B830002F2003F0C7FE00E004E0BDE8F05F112018
:10B84000FDF762BFBDE8F05F05F0C0BFBDE8F09F47
:10B85000401F0020041501400010014073B58CB05A
:10B860000646002000900D9880B100246D462146C8
:10B870000DA802F084FA30B1009805EB40008480F6
:10B880000098401C0090641C142CF0D32C226946B4
:10B890003046FDF7EBFD0EB070BD2DE9F041178885
:10B8A0000646B81D14460D46984202D90C20BDE844
:10B8B000F0813188072206290AD34FF4486C4FF6ED
:10B8C000FF73614501D9994202D17088062801D2DF
:10B8D0001046ECE7604501D99842F9D1994203D06E
:10B8E000984201D08142F3D80520E85520881221E2
:10B8F000401C80B2208029542088401C80B22080C7
:10B900004119308806F04EFE2188084480B220801C
:10B910004119708806F046FE2188084420800020E6
:10B92000C5E7FEF78FBA000038B54A7A0F4B62B10F
:10B9300000220A725969002906D001228DF80020E0
:10B94000ADF802006846884738BD0A7A62B19B6844
:10B950004C68024619462046FEF742FB0028F3D009
:10B96000BDE8384006F016B95B68F1E7EC2200202C
:10B97000F0B585B016460F4604461D4614220B4905
:10B980006846FDF773FD0A488DF80870ADF802406F
:10B99000ADF80A608DF80C50017800222046FEF7C1
:10B9A000F9FF684600F08AFC05B0F0BDC82D020022
:10B9B000D81E00200A2A01D00C2070470A88028075
:10B9C0008A788270CA78C2700A7902714A794271A3
:10B9D0008A798271CA7902720A7A82724B7A027B00
:10B9E00063F3000202734B7A5B0863F34102027354
:10B9F0004B7A9B0863F382020273497AC90861F3A8
:10BA0000C302027300207047FEF71CBA70B5464EA1
:10BA100005460324308845A104EB004003F092F969
:10BA2000308846A104EB004003F08CF9287B45499F
:10BA300051F82020308844A104EB004003F086F93F
:10BA4000EA793088002A04EB004064D043A103F077
:10BA50007DF93C49A879203151F82020308844A153
:10BA600004EB004003F072F9AA883088002A04EB46
:10BA7000004054D043A103F069F9308846A104EB9B
:10BA8000004003F05FF930882A7A04EB004044A1BB
:10BA900003F05CF930886A7A04EB004044A103F0BB
:10BAA00055F93088AA7A04EB004045A103F04EF91D
:10BAB0003088AA7B04EB004045A103F047F93088A9
:10BAC0004BA104EB004003F03DF9287C4DA1C0F3ED
:10BAD000C002308804EB004003F038F9287C4FA105
:10BAE000C0F38002308804EB004003F02FF9287C7B
:10BAF00050A1C0F34002308804EB004003F026F967
:10BB0000287C52A100F00102308804EB0040BDE81F
:10BB1000704003F01BB953A103F014F999E757A142
:10BB200003F010F9A9E70000782000200D0A437502
:10BB30007272656E742054696D653A000D0A446135
:10BB400074653A00201E002009446179206F662048
:10BB50007765656B2020202573000000094461791A
:10BB6000206F66206D6F6E746820202569000000CC
:10BB7000094D6F6E7468206F6620796561722025AB
:10BB800073000000095965617220202020202020C8
:10BB900020202025690000000D0A54696D653A00D7
:10BBA00009486F757273202020202025690000004D
:10BBB000094D696E757465732020202569000000A9
:10BBC000095365636F6E64732020202569000000AF
:10BBD000094672616374696F6E732025692F32356F
:10BBE00036206F662061207365636F6E640000000D
:10BBF0000D0A41646A75737420726561736F6E3AE1
:10BC00000D000000094461796C69676874207361F4
:10BC100076696E6773202578000000000954696D0D
:10BC200065207A6F6E652020202020202020257836
:10BC3000000000000945787465726E616C207570B3
:10BC4000646174652020257800000000094D616E54
:10BC500075616C20757064617465202020202578E2
:10BC60000000000009446179206F66206D6F6E74DA
:10BC7000682020556E6B6E6F776E00000959656104
:10BC80007220202020202020202020556E6B6E6FF7
:10BC9000776E000010B5044680898A8886B090428D
:10BCA00036D1C888002833D1CA8901A81031FFF7DE
:10BCB00081FE042130BBBDF8040042F20F729042B5
:10BCC00020D840F22E62904200D2D8B99DF80600EA
:10BCD0000C2817D89DF807001F2813D89DF80800D6
:10BCE00017280FD89DF809003B280BD89DF80A00AB
:10BCF0003B2807D89DF80C00072803D803208DF8AF
:10BD0000000001E08DF80010226869462046904747
:10BD100006B010BD01460148FEF7CABE58210020FA
:10BD200030B5044685B000211B4805F086F8002890
:10BD30002FD00025204600F040FF68B1112812D016
:10BD400086281BD0A0F54051023903D00146204679
:10BD500005F028FF294607E005B029462046BDE842
:10BD6000304001F0F5BC0121204601F0F1FC05B0A6
:10BD70000021BDE83040084805F093B81422074977
:10BD80006846FDF773FBADF80240684600F072FAB2
:10BD9000E0E705B030BD0000A51E00203C2D0200EC
:10BDA0007FB50C4610B1012004B070BD207900268B
:10BDB00038B141F61D5501281BD0022826D00F208E
:10BDC000F2E70220207102960396E068019069462E
:10BDD00001A805F03BFC50B102988188E180008801
:10BDE0002081BDF80010029805F0AEFCDCE70A20C7
:10BDF000DAE70A4B6A460021A01D05F0E3FB38B1E3
:10BE0000064918398E61CE610A28CDD12846CBE784
:10BE100002488188019805F097FCF5E7801F002013
:10BE20002DE9F843054690F8C6020F4600EB800165
:10BE3000C1EB801005EB400695F8C542914604EB36
:10BE4000C40006EB40013279601C0A31904226D1D1
:10BE50006B460022284601F0B3FA18B310E0401EEA
:10BE6000A04201D1002004E004EBC40006EB400036
:10BE70001C30804602466B46284601F0A1FA30B1DC
:10BE800000203870694648469EDFBDE8F88395F883
:10BE9000C5024146401C641C85F8C502E4B23079F5
:10BEA000A042DCD8012038700020EEE72DE9F047F1
:10BEB0000025DFF88C803CE06068002100EBC506BF
:10BEC000012032789146FDF7BEFAD4E9062300EA54
:10BED000020701EA030C57EA0C0728D082438B4380
:10BEE0004846C4E9062303F02FFC32788246914687
:10BEF00001200021FDF7A7FAD4E9042300EA020497
:10BF000001EA03074A4650460021FDF79CFA4440E7
:10BF10004F403C430BD17078012801D0012100E053
:10BF20000021726881EA0A010AB1484690476D1CF7
:10BF3000EDB298F8000044468542BDD3BDE8F087D5
:10BF4000101F00202DE9F047894690F8C612904650
:10BF500001EB8102C2EB811100EB4107384605F08D
:10BF60000FFC06002FD0194CA06806282BD2184DC4
:10BF7000762205EBC0103946A0F80280001DFDF7BF
:10BF800075FA0027B9F1000F04D0A06805EBC010C6
:10BF9000077004E0A168022005EBC1110870A068D9
:10BFA00005EBC011401CCE67A060E16888420AD151
:10BFB000002604E005EBC610C16F8847761CE068D8
:10BFC0008642F7D3A760BDE8F0870000941E0020EA
:10BFD0009823002070B50E4690F8C612154601EB66
:10BFE0008102C2EB8111A0B000EB410005F0C8FB5B
:10BFF000040009D07C2205496846FDF737FAADF800
:10C00000025068460196A04720B070BDAC2C0200DB
:10C0100070B50E4604464FF43371FDF740FA1148EF
:10C020000025A4F8CA62856084F8C9520E4884F8D5
:10C03000C65284F8C552006820602246012130466D
:10C040009BDF0121112806D0002809D184F8C712EE
:10C0500084F8C85203E084F8C71284F8C81200209C
:10C0600070BD0000941E00208023002010B5002128
:10C07000024801F0BDFE80F3100010BD68310020C1
:10C080000E4910B50A784C780023A24212D0521CF7
:10C09000D2B20A70022A00D10B70084A0B780C3217
:10C0A00052F8232002608868104420F07F408860A6
:10C0B000012010BD0360002010BD0000401F0020C3
:10C0C00013460A460021FFF753BC00002DE9F84350
:10C0D000104D0F4680461E4691466946286801F07D
:10C0E000E2FD040014D01C21FDF7D9F901202071D4
:10C0F000C4F81490380BC4F80080C4E902606946A3
:10C10000286801F0F1FD05F0F1F90020BDE8F883A1
:10C110000420FBE7942E020010B503780022072BC1
:10C1200006D2DFE803F005040610202930000A706B
:10C1300010BD01230B7003898B818388CB81C0687C
:10C1400088600A7410BD02220A7002898A8182887E
:10C15000CA81C2688A60807D062802D000200874E7
:10C1600010BD0120FBE703220A70C2888A81028980
:10C17000CA81C068886010BD04230B70C0888881A4
:10C18000CA818A6010BD0520087010BD70B5064DCB
:10C190000646002455F8241009B130468847641C2F
:10C1A000042CF7D370BD0000CC2A002030B5044623
:10C1B000006887B00D46806800281FD018216846A7
:10C1C000FDF76DF90195A0680590207910B101285F
:10C1D00010D107E001208DF8000020690290E0688E
:10C1E000039005E002208DF80000E0680003029053
:10C1F00060690490206881686846884707B030BD50
:10C2000070B586B015460C00064619D0112C17D013
:10C21000082C15D014216846FDF741F9ADF80260ED
:10C22000304600F0DDFEADF804000D2C0AD0862C5F
:10C230001CD007208DF800000294684600F04CF8EE
:10C2400006B070BD03208DF8000025B12878C00726
:10C2500001D0012000E002208DF8080000208DF8B8
:10C260000C0041F20110ADF80A00E6E706208DF857
:10C270000000E2E710B50446408800F0B1FEA0805F
:10C28000024801682046BDE810400847AC1E002067
:10C290002DE9F04107460024064E074D05E000BF9A
:10C2A00056F8241038468847641CE8788442F7DB47
:10C2B000BDE8F081A8280020C81E002010B5044663
:10C2C000408800F08DFEA080024801682046BDE84D
:10C2D000104008479C2D02000149096808470000EA
:10C2E000F02D020070B586B0044614216846FDF7B3
:10C2F000D6F8A0890125A0F54040ADF804002078CB
:10C300002A4E062833D2DFE800F0320303032C481C
:10C31000A08900F0BDF930B9E08943F6FE71A0F5BF
:10C320004040884223D8A07B8DF80800207803285D
:10C330000FD000208DF80900A0680390606850B10C
:10C3400009208DF8000060680490684604F0F2F857
:10C350000DE00120EEE708208DF800008DF8105068
:10C36000F3E7A08900F094F908B1E08930B1707862
:10C37000002801D004F00EFA06B070BD606820B14C
:10C380000B208DF800007570DFE70A208DF80000A3
:10C39000BDF8040004F088FAF5E713208DF80000DA
:10C3A0004FF6FF70ADF80400CFE70000B81E002084
:10C3B00038B504460E480078A8B1A4F57F40FF3890
:10C3C0000FD0684604F0C4FF78B105210170012147
:10C3D0000171C480684604F0C9FF05F079F80020B7
:10C3E00038BD042038BD022038BD082038BD00000B
:10C3F000881F00200C4808B5007888B1684604F012
:10C40000A7FF78B106210170684604F0AFFF074826
:10C41000017809B10121017305F05AF8002008BD27
:10C42000022008BD082008BD881F0020902B002096
:10C43000F0B587B014216846FDF731F82B4C207811
:10C4400018B16846FFF7A2FE4EE0201D01F0B2FCD5
:10C45000B8BB4FF010204169000400694A1C02D1AA
:10C4600000EB40000101224800220161A1F540518A
:10C47000C160204902F030F8002820D11F481C2359
:10C480008C221D49006801F0FBFB03F043FE050010
:10C4900014D0022D12D000270126062D12D005A897
:10C4A00004F056FF88B106700C2D18D2DFE805F0B5
:10C4B000170F170F17161716171113110B2007B0A8
:10C4C000F0BD11E026706760BBE70820F7E7077151
:10C4D00005E0032100E00221017100E0067105A8DA
:10C4E00004F044FF04F0F4FF0020E8E7881F002078
:10C4F00030200020A42E0200DC2A00200C2E020096
:10C5000038B5040014D0694605F0A0F8A0B1BDF814
:10C51000000000EB8001094800EB8100C16849B1CF
:10C52000A17A39B1C168491EC1600020A07238BD2E
:10C53000052038BD062038BD0A2038BD682B0020F4
:10C540001FB501A9684605F03DF804B010BD07B558
:10C5500013460A466946002005F034F80EBD07B5BB
:10C5600013460A460021684605F02CF80EBD20B19E
:10C5700019B100680860002070470520704700006E
:10C58000F8B50D46040018D0BDB1694605F05EF857
:10C59000A8B1BDF800000B4900EB800001EB800062
:10C5A00001210C30666801F008FC2E6060680C30D8
:10C5B00068600120A0720020F8BD0520F8BD0A20A7
:10C5C000F8BD0000682B002018B10323002206F0FC
:10C5D00029BA052070470223002206F023BA12B1BF
:10C5E000022306F01FBA052070470000084910B565
:10C5F0000A69042A0AD0074A096942F82100044856
:10C600000121103001F0D9FB002010BD0C2010BD1D
:10C61000681F0020CC2A002038B5044609480D4682
:10C62000007858B164B16946284606F0F5FA00284A
:10C6300003D1BDF800102180658038BD022038BDCF
:10C64000052038BD881F002010B504460E4800782C
:10C6500098B1A4B12188022913D80C4A01EB8100BA
:10C6600002EB800260885289C31C934209D806F00D
:10C67000C7FA00202080608010BD022010BD052078
:10C6800010BD042010BD0000881F0020682B002072
:10C6900043F6FE71A0F54040884201D80120704762
:10C6A0000020704710B504460078182802D1FEF724
:10C6B0004DF9207010BD10B504460078182802D13D
:10C6C000FEF744F9207010BD70B50D460446B0F871
:10C6D0009810D0F894000122FDF783FE00B1057098
:10C6E00004F13C0204F1940104F1540072DF70BDC6
:10C6F00070B51346002206461546862902D0112938
:10C7000002D002E0012200E001250D4C73B1A179B5
:10C71000FEF740F92A4661793046FEF73BF90022E0
:10C72000A1783046FEF736F9002203E0A178FEF743
:10C7300031F92A4661783046BDE87040FEF72AB9E3
:10C74000E01E0020F7B517460E0011D00098002516
:10C7500060B100242146684601F011FB18B1A0B277
:10C760003946B0476D1C641C142CF3D32846FEBD1B
:10C770000020FEBD406804F00BBE000070B508B19B
:10C78000012070BD194C0025207B08B1257301E004
:10C7900000F0A0F82078082826D2DFE800F0250471
:10C7A000080C10251420BDE8704000F021B8BDE849
:10C7B000704000F07DB8BDE8704000F05FB8BDE8A3
:10C7C000704000F03BB86088084900EB80002839D1
:10C7D00001EB80004068BDE8704003F07BBC656001
:10C7E000BDE8704003F084BC0F2070BD902B00208A
:10C7F0001149F0B48A1C00200346A1F128050C1849
:10C80000A67A4EB1A37200EB800405EB8404E668BF
:10C8100016B9247C012C0AD0401C80B20228EED329
:10C820000B704B804B60F0BC41F61D507047108080
:10C83000F0BC00F03DB80000902B00200C4841886F
:10C8400001EB8102A0F1280101EB8201CA6852B11B
:10C85000052101700748022181800168002301221F
:10C86000054801F0A3BD042202704968F6E7000004
:10C87000902B0020901F00203020002038B50A495E
:10C88000084803240B684268898803EB81015388B8
:10C890000470DB1C00201B0400909B0B034801F07C
:10C8A000F5FE38BD902B0020901F00203020002086
:10C8B000074910B54888091D04F018FF18B1BDE8F4
:10C8C0001040FFF7DBBFBDE81040FFF7B7BF000027
:10C8D000902B0020F0B51F481F490125067802243F
:10C8E0008B88A0F12802082E19D2DFE806F0041880
:10C8F000181B222F2F170189491C0181002141801B
:10C9000080F80C1001EB810312F8233043B10023AF
:10C910004418491C89B2A3720229F3D30570F0BDF3
:10C920000123F5E742685288D21C1A448A800470B9
:10C93000F0BD46880D6806EB860602EB8602566857
:10C940000E60556013818C80062100E00721017084
:10C95000F0BD0000902B0020901F002010B5018832
:10C960008288502905D0522914D1104600F0BCFE0F
:10C9700010E0017B01290DD1817A01290AD10089BA
:10C98000A0F52451023905D10121104600F0E0FE46
:10C9900005F078FE044800220249C078BDE8104046
:10C9A000FDF794BF8DA10100A41E0020017800298D
:10C9B00002D1408800F098BE7047000010B5124CBC
:10C9C00000202070FDF7C2FFA070FDF7BFFFE070F0
:10C9D000FDF7BCFF2071FDF7B9FF6071A178182940
:10C9E0000FD0E17818290CD02179182909D01828FE
:10C9F00007D00121601C04F019FA012020700020EA
:10CA000010BD032010BD0000A41E002010B5017849
:10CA1000082916D1417AA1B9017A072902D008293B
:10CA20000FD10AE0808800F0C5F9A0F57F41FF39F9
:10CA300007D0012100F08CFE03E00021034804F040
:10CA400030FABDE8104005F01DBE0000A51E002014
:10CA500010B504460A4841782046FDF783FF68B1C7
:10CA60000848002101EB410200EB82025288A242F9
:10CA700001D1C8B210BD491C1429F3D3FF2010BD49
:10CA8000B41E00209826002070B5094D094E0024E0
:10CA900004EB440005EB800071784088FDF762FFED
:10CAA00020B1641C142CF3D3FF2070BDE0B270BD24
:10CAB00098260020B41E00202DE9F0418046024651
:10CAC00001200021FCF7BFFC1A4F05460E4678688E
:10CAD000FDF7CAFA00280CD1174CD4E906211046FC
:10CAE0002A4001EA06031A4305D0A843B143C4E92A
:10CAF0000601BDE8F081404602F026FE30B1D4E9DF
:10CB0000040128433143C4E9040105E0D4E90410D9
:10CB1000A943B043C4E90410D4E9060128433143D2
:10CB2000C4E90601A1687868BDE8F0410022FDF77C
:10CB300057BA0000FC2D0200101F002003484FF6DA
:10CB4000FF7141800121017000207047B01E00205C
:10CB50002DE9FC41804600F043FA0024032501271B
:10CB6000A0F57F412646FF3908D06A46082103F028
:10CB7000F9FB18B90198841D8688056832462B4652
:10CB800021464046B1DF042804D0082804D00B28F1
:10CB900008D002E0112000E00020002F00D10B207F
:10CBA000BDE8FC810027A80701D50125E6E734434D
:10CBB000F5D0002426460325E0E72DE9FC41804618
:10CBC00000F00EFA0646A0F57F40FF380ED0012592
:10CBD0002A466D1C0027ADB26B460821304603F093
:10CBE000EBFB040006D0072C25D025E043F2020021
:10CBF000BDE8FC81019903230A1D0B604046891D95
:10CC0000B2DF040004D00C2C09D0052C09D009E0B7
:10CC100032460821104603F045FC04460CE001278B
:10CC200000E000240821304603F028FC00B1032472
:10CC3000002FCDD100E00C242046D9E7428800EB3C
:10CC400082020C328A4201D9022070478188A1F504
:10CC50007F42FF3A03D0008808B1002070470120CE
:10CC60007047884204D20068401C01D00120704700
:10CC7000002070473EB5027802230C46B3EB520FFA
:10CC800017D1B0F80110ADF80010C1788DF802107E
:10CC90008188ADF8041080798DF8060002AA01A9F8
:10CCA0002046FDF711F8032202A96846FCF709FCAB
:10CCB00008B100203EBD01203EBD000010B50C466D
:10CCC000FFF7C6FEFF280CD0074900EB400001EB40
:10CCD0008000416821600189A180807AA0710020D4
:10CCE00010BD052010BD00009826002070B50188F9
:10CCF00090B0102959D1011D28226846FCF7B6FBD7
:10CD00009DF804004FF6FF76032134466D46B1EBE3
:10CD1000500F2AD003F07CFC9DF8040040080ED090
:10CD200001280CD0022820D118E00C99281D1131BF
:10CD3000FCF7F3FE18B100BFBDF8284015E00BAAC0
:10CD40000AA9072003F038FC0028EED10DE00C9969
:10CD5000281D491CFFF78EFF0028EDD10BAA0AA958
:10CD6000072003F029FC0028F1D1BDF80000291D9F
:10CD700000F030FFB44218D0BDF80000214600F0AA
:10CD800019F9BDF80000ADF82A000020ADF82C40DC
:10CD9000074E8DF828000AAD044600BF56F824104F
:10CDA00028468847641C022CF8D310B070BD0000E0
:10CDB000502D0200094A002101EB410332F82330D3
:10CDC000834205D101EB410002EB800040887047AF
:10CDD000491C1429F0D34FF6FF70704798260020A5
:10CDE0002DE9F041CEB00D46070019D0C5B10DF1C7
:10CDF000B8085020CDE94B80B8216846FCF74FFBBE
:10CE0000002042A94FEA0D06C0EBC00202EB00125F
:10CE1000324441F82020401C0828F5D300242BE0A0
:10CE20000022114610466FDF4EB0BDE8F081502160
:10CE30002EA8FCF734FB37F814004CAB4AAA0721A4
:10CE400003F0EEFB05280AD0072808D09DF8C9009A
:10CE5000400806D0012804D043F20220E4E7052070
:10CE6000E2E7C4EBC40000EB04103044172208F1E1
:10CE70000101FCF7FBFA641CAC42D8D3EAB20021F2
:10CE800042A86FDFD0E73EB50C46054603F0C0FB75
:10CE90000BE0BDF80000A04207D02846029900F040
:10CEA0002FF810B1BDF800003EBD01AA6946072069
:10CEB00003F082FB0028ECD14FF6FF703EBD00006E
:10CEC00010B50D4C18200D4A607000204FF6FF7110
:10CED00000EB400302EB8303401C59801428F7D376
:10CEE000FDF734FD6070182803D001202070002069
:10CEF00010BD032010BD0000B41E002098260020A5
:10CF00002DE9F0410C46054600F1110701F111062B
:10CF10001022491C401CFCF7D4FA48B9681C00F0E8
:10CF200075FA28B1601C00F071FA08B1012400E024
:10CF3000002431463846FCF7F0FD3B780222B2EB84
:10CF4000530F0CD00321B1EB530F08D03378B2EB61
:10CF5000530F04D0B1EB530F01D0012100E00021A9
:10CF6000084201D18C4302D00120BDE8F0810020AD
:10CF7000FBE7018811B9421892780AB10120704785
:10CF8000491C0829F7D30020704710B50C4603460A
:10CF9000FFF7EFFF00280AD018882188884205D1C2
:10CFA0000822A11C981CFCF78CFA08B1002010BDC7
:10CFB000012010BD03F0CCBC70B50446FFF7FAFEAB
:10CFC0000546204603F0D1F94FF6FF7104468D4225
:10CFD00003D014B9284603F0BBFC204670BD000006
:10CFE00010B5FFF735FDFF2805D0044900EB4000E0
:10CFF00031F8200010BD4FF6FF7010BD98260020BC
:10D000003EB5044603F004FB0EE00199204646318C
:10D01000FFF7BBFF28B9019920462A31FFF7B5FF7A
:10D0200010B1BDF808003EBD6A4602A9072003F012
:10D03000C3FA0028E9D14FF6FF703EBD7CB5144617
:10D040000A000A49897802D015688D4203D323B1BA
:10D050001D688D4201D204207CBDCDE900431346FA
:10D060000246034803F0B8FC7CBD0000B41E00205B
:10D070008827002070B50C4606469AB01021184843
:10D08000FCF70DFA174800252EB324B38470620014
:10D0900031461348FCF7EAF9382102A81895FCF745
:10D0A000FEF9009518AB02AA21463046019503F01F
:10D0B00093FC00280DD110AA0DF10801C0EBC003AC
:10D0C0000B4442F82030401C0828F7D3E1B2104648
:10D0D0006EDF1AB070BD8570002108466EDFF8E77C
:10D0E00088270020B41E002010B50A4941600A4874
:10D0F00000F060FE58B902F0A5F907491C238C2204
:10D10000087404488C39001F006800F0B9FD002045
:10D1100010BD0000982E02002C2C00202DE9F041BB
:10D120002D4F002518B17D600120BDE8F081087900
:10D13000012258B1294E01280CD0274C4FF002088B
:10D140000834022821D0032842D128E00A7102F0D5
:10D15000CFFF3BE05FF0000000EB800116F82110EC
:10D16000022908D0401C80B20228F5D33A707D60B5
:10D1700041F61D50D9E700EB800006F8205006EB81
:10D180008000406802F0A6FF20E00D71A4F8048042
:10D19000002301221248216801F008F916E00D7100
:10D1A000206802F097FF0D4923682831498801EB78
:10D1B000810206EB8201D1F804C0C4F800C04B60C4
:10D1C000A3880B81A4F8048006F822500028ACD074
:10D1D0007D600E20A9E70000881F0020682B00203A
:10D1E000302000200146034802888A4200D00020F7
:10D1F00070470000D82200202DE9FC5F0E00834616
:10D20000DDE90C47C6F1000098469246814600D4FD
:10D210000846012503E000BF90FBFAF06D1C504565
:10D22000FADAA84500D9454624B1002E01DB78077B
:10D2300000D5641EB80702D5B8F1000F0AD0F80770
:10D2400008D13CB1A54205D220215846641EFEF704
:10D25000F7F9F6E7002E02DA4E462D2102E07807B4
:10D2600003D52B215846FEF7EBF907F003000228FF
:10D270000BD1B8F1000F08D13CB1A54205D2302145
:10D280005846641EFEF7DCF9F6E7CDE90047434651
:10D2900052463146584605F09BF9BDE8FC9F000018
:10D2A00070B50D46044600684FF4887102F04FF9DE
:10D2B0004FF49071206802F04AF94FF4927120689F
:10D2C00002F045F94FF4A271206802F040F920689D
:10D2D0001249C0F8041320686907000B40B2090E18
:10D2E000002806DA00F00F0000F1E02080F8141D9D
:10D2F00003E000F1E02080F8001420680121000B19
:10D3000040B200F01F0291404009800000F1E0208F
:10D31000C0F88012C0F8001170BD000010030200B8
:10D32000024600201268930702D0530702D47047C8
:10D33000500714D502F00300012802D002280CD1B6
:10D3400005E0C2F383100B68801C184404E002233C
:10D35000086803EB92521044086001207047086887
:10D3600000EB9253C2F38910401CEEE70248007AAA
:10D37000002800D0012070472C2C0020F0B58488B4
:10D38000A518944200D82246A41AC288D6189A42F8
:10D3900000D81346D21A4B880788BB420CD340886A
:10D3A000834209D88888A04206D3A84204D8C888F6
:10D3B000904201D3B04201D90020F0BD0120F0BD60
:10D3C00010B509892AB1D088491C814218D10020A2
:10D3D00010BD90F8C62202EB8204C4EB821200EB6F
:10D3E000420212899142F2D0491C198090F8C6126B
:10D3F00001EB8102C2EB811100EB4100008902E0E8
:10D400001980D088401E5880012010BD0021425C48
:10D410000AB101207047491C1029F8D30020704739
:10D42000800701D000207047012070470A4810B5DE
:10D43000807860B1002401E0022C06D02046FDF780
:10D4400051FE641C042CF7D310BD0324F6E7BDE89D
:10D450001040FDF767BE0000741E002003480179EC
:10D46000C90702D00078FDF7C3BF7047741E0020C3
:10D470001721018041800021017141717047000036
:10D480002DE9FE4F2B4D984691460F00824601D064
:10D4900000260DE0684600F0C9FB6A4600215046B0
:10D4A00002F0CFFE2878009E10B99DF8090098B1CF
:10D4B0004A463146504604F06DFD044601460022BE
:10D4C0005046FFF715F90D2C32D008DC84B3082C38
:10D4D0002ED00B2C0BD12BE00520BDE8FE8F112C9C
:10D4E00010D0862C1AD0A4F54050023820D0032545
:10D4F000B8F1000F04D0324621465046FEF780FEB8
:10D500002846EAE73A4629795046FDF743FA4A4663
:10D51000E9785046FDF73EFA0025E9E73A462979D1
:10D520005046FDF737FA4A46E9785046FDF732FA99
:10D530002546DDE7E01E00202DE9F041204F0E4694
:10D54000154604463978FDF70DFA002835D02046F7
:10D5500002F06EFE50B32046FFF742FD80462046A3
:10D56000B978FDF7FFF908B1012700E0022720464E
:10D5700003F006F90028404602D0FFF71DFD0DE03C
:10D58000A8F57F41FF3909D0072102F077FF01009C
:10D5900004D0052902D0204604F018FB2B46324661
:10D5A00039462046BDE8F041FEF7E2B92A46314649
:10D5B0002046BDE8F041FEF783BDBDE8F0810000E4
:10D5C000D81E002070B5094D0646E978FDF7CAF966
:10D5D000044629793046FDF7C5F901462246304612
:10D5E000BDE870400123FFF74BBF0000E01E0020A4
:10D5F0002DE9F047394E002780463D46DFF8E090A0
:10D60000D6F804A057E003D00446D0F81C8035E0DB
:10D6100099F8002002EB4201521CD2B289F8002096
:10D6200009EBC10199F80230091D9A4201D189F82C
:10D63000005048680A780446012A12D0022A02D013
:10D64000032A3BD108E004F055FE00B10127257400
:10D6500034E00574C06900E070680028F9D170609A
:10D660002CE0207C50BB88686060C868A0600869B6
:10D67000E0604869A061F07800B165606268B168F7
:10D68000184B501A20F07F40984202D2A1680844FB
:10D6900006E0881AA16820F07F40814202D9081A6A
:10D6A000206000E0256065600120A56020742046B0
:10D6B000E56104F001FEB8F10000A4D199F8001072
:10D6C00099F801008142A3D117B97168514502D080
:10D6D0000120BDE8F0870020FBE70000401F00208C
:10D6E000A8290020FFFF7F0030B585B00546002443
:10D6F00014216846FBF7D3FEA5F57F40ADF8025034
:10D70000FF3815D02846FFF723FA98B10B2815D01B
:10D71000112811D0A0F54051023903D00146284606
:10D7200004F040FA09482246C1782846FDF732F94C
:10D7300005B030BD0E2002E00124F3E70F208DF884
:10D7400000006846FEF796FDECE70000A41E0020EE
:10D750000A4602498978FDF71DB90000A41E002081
:10D76000F8B5054600780C46002620420FD100206F
:10D770008DF800006846FCF787FC2878204202D12B
:10D780002043287001269DF80000FCF7A1FC3046DC
:10D79000F8BD00002DE9FF410026234800F007FBFB
:10D7A0002148001F074600F002FB204C60680090F3
:10D7B000A56800E000986946284004EB80000C3022
:10D7C000FFF7AEFD0028F5D101AA009901EA050393
:10D7D00004EB8303491CDB6842F82030401C0091B5
:10D7E0000228F2D3019800F0030001280BD0022890
:10D7F00010D10198032101EB90500099BDF80A6007
:10D8000001EB900005E00198BDF80A60C0F38310B9
:10D8100008440090384600F0C7FA08B100986060EC
:10D8200004B03046BDE8F081643100204C2D00206A
:10D8300088B04FF40041002001F0F6FA08B1FCF77F
:10D8400001FB01F061F9FCF7A1FB08B1FCF7FAFA62
:10D850005E4A00215E48FCF787FB08B1FCF7F2FA4C
:10D860005C490320FDF77AFD08B1FCF7EBFA694645
:10D870000020FDF77BFC08B1FCF7E4FA9DF80000FE
:10D8800002287DD00025544A0A210820FCF756FBC7
:10D8900008B1FCF7D7FA01F0E5FB08B1FCF7D2FAC2
:10D8A00001F076FD08B1FCF7CDFA002469460120AD
:10D8B000009401F001FC08B1FCF7C4FA684601F0DD
:10D8C00079FC08B1FCF7BEFA9DF8080043A120F0EE
:10D8D0000F00401C20F0F00010308DF808000A22E4
:10D8E00002A87CDF08B1FCF7ADFA4FF4C8700094D1
:10D8F0000194ADF800004100ADF80440ADF8060019
:10D90000ADF8021068467ADF08B1FCF79BFA32489E
:10D910000021C03000F0E1FA08B1FCF793FA324878
:10D92000FDF73AF908B1FCF78DFAFCF737F903F087
:10D930001DF82E480094CDE90140274802A9D030B7
:10D9400000F05DFB08B1FCF77DFA294800902948FA
:10D95000019021486946B030FDF75EF808B1FCF748
:10D9600071FA1C216846FBF79AFD4FF42030CDE98F
:10D9700000404FF47020032602908DF80C6000E008
:10D9800021E01D4805901D480690ADF80E408DF829
:10D9900010406846FCF756FF08B1FCF753FA1848E8
:10D9A00018A1008806EB004001F0CCF92846FCF7EE
:10D9B0002FF900BFFCF7A2FA01F0B4F80028F9D162
:10D9C00001F064FBF6E701255DE70000391B02006A
:10D9D000742C020061B20100A82000204E6F726416
:10D9E00069635F435453000015BD0100A1F00100BD
:10D9F00091FC010009BA0100F1FB010023B901000B
:10DA00007820002043757272656E742054696D65CC
:10DA1000207365727669636520636C69656E742036
:10DA2000737461727465642E0000000070B5144652
:10DA300082880E4605462088111D0144921C994299
:10DA400001D8FE2A01D90C2070BD521C3254208806
:10DA5000FF21401C80B2208031542088401C80B2BD
:10DA600020808119288804F09DFD2188084480B217
:10DA70002080AA8842B1A96841B13044FBF7F6FC86
:10DA80002088A98808442080002070BD072070BD30
:10DA90002DE9F047C7880446181D16468946B0FB95
:10DAA000F7F1B0FBF7F207FB12009A193A44D21CC7
:10DAB000B2FBF7F2DDF820A001E02468491E00293E
:10DAC000FBD13D1A8846B54216D818E0BAF1000FCE
:10DAD00005D0211809EB08002A46091D04E020445E
:10DAE00009EB08012A46001DFBF7C0FC0020246852
:10DAF000761BA844B74201D9354600E03D46002ECA
:10DB0000E4D1BDE8F087000030B5024659B101F01C
:10DB1000B7F90021074C09E004EB810315685B8825
:10DB2000AB4202D11160002030BD491C8142F3D3C9
:10DB3000052030BD44200020F8B50F46017814467A
:10DB40000546012901D1687830B12088821C9A42AB
:10DB50002DD8012902D006E00720F8BD69780144DC
:10DB6000891C994223D8181A801E86B2ADF800602D
:10DB70002188B81C084469467DDF0028EDD128784B
:10DB8000022805D1BDF80010B14201D809210AE0F0
:10DB90000821012805D16878B04202D8ADF800000C
:10DBA00001E0ADF80060BDF80000FE2801D90C20AE
:10DBB000F8BD2288401CB8542088401C80B22080C8
:10DBC00039542088401C2080BDF800100844208073
:10DBD0000020F8BD70B505460C004FF0FF0020D0C6
:10DBE0004FF6FF76B5421CD00E48012241782846F8
:10DBF000FCF7D0FE2846FEF72BFFFF2803D1FEF7E7
:10DC000043FFFF280DD0084B00EB400203EB8201DD
:10DC10004D8023F8226022684A60A2880A81A27996
:10DC20008A7270BDB41E002098260020034A00218D
:10DC30009268C0E90021816070470000E01E00206A
:10DC400070B54FF6FF750E46A84201D1002000E0E6
:10DC5000401C84B208E02146304603F016F908B1B2
:10DC6000204670BD641CA4B2FF2CF4D9284670BDB8
:10DC700010B5FBF71AFB08B1002010BD112010BD34
:10DC800010B531B1B2FBF3F403FB14241CB109202D
:10DC900010BD0E2010BD01600021416081608281B5
:10DCA000C381084610BD70B50C460546FBF7B2FAB5
:10DCB000002802D021882868084470BD10B50A8861
:10DCC00049888A4203D1FBF7E7FA012010BD002002
:10DCD00010BD70B50C460546FBF7C1FA002802D00E
:10DCE00061882868084470BD10B50A8849888A424E
:10DCF00003D1FBF7ABFA012010BD002010BD01F0ED
:10DD00001F0301229A40D243490900EB81001146CA
:10DD100000F059B80A4601F01F030121994010B5DF
:10DD200052090C4600EB820000F05DF8204000D064
:10DD3000012010BD2DE9F04180460D460024481E0B
:10DD4000012101EB501716E058F82400C04390FA67
:10DD5000A0F0B0FA80F020280CD200EB4416AE42BE
:10DD600008D231464046FFF7D5FF0028ECD13046B7
:10DD7000BDE8F081641CA742E6D82846F8E74A09C6
:10DD800050F8220001F01F0201219140084000D00C
:10DD90000120704701F01F0301229A40490900EB5E
:10DDA0008100114600F029B8002100F017B80121C8
:10DDB00000F023B8012100F016B808B56A46FBF759
:10DDC000C0FA009808BD08B56A46FBF7A0FA0098AB
:10DDD00008BD08B56A46FBF7B4FA08BD08B56A463F
:10DDE000FBF795FA08BD08B56A46FBF783FA08BD4C
:10DDF00008B56A46FBF772FA08BD08B56A46FBF734
:10DE000079FA009808BD08B56A46FBF7A7FA0098AA
:10DE100008BD38B5044600258DF800506846FCF76B
:10DE200033F921686268086890420ED9401E086084
:10DE30000178A38AE26801FB0325227A2168101A7F
:10DE4000C0B20A79824200D208719DF80000FCF746
:10DE50003FF9284638BD38B5054600208DF800004A
:10DE60000C466846FCF710F9E868A98A201AB0FB4E
:10DE7000F1F12A681068431C136001709DF80000DE
:10DE8000FCF726F938BD10B530B1017A4268036855
:10DE9000891AC9B21A6006E00E2010BD03681A681C
:10DEA000541C1C601170491EC9B2F7D200680021D1
:10DEB0000171084610BDC20800F007030120895C0B
:10DEC00098400840704710B5C20800F00703885C0E
:10DED00001249C402043885410BD10B560B1C1603E
:10DEE000172120F8021B20F8021B1B2100F8021B3F
:10DEF000FFF7BEFA002010BD0E2010BD7CB50C4609
:10DF00008188002933D102880025102A06D0112AE1
:10DF100009D03A2A0BD0552A2ED129E001462046B5
:10DF200001F074FE28E0A01DFFF7A2FA24E02246CB
:10DF3000408934F8063F834200D81846608017288D
:10DF400000D217206080D06878B1607968B1174B33
:10DF5000D3E90003CDE90003ADF802106088ADF805
:10DF60000400D368694610469847657125717CBDE9
:10DF70000146204601F090FFA07A0028F7D02846FD
:10DF8000E188A5DF012670B11128F0D001F0D0FAA8
:10DF90000246074807A1008802B006EB0040BDE832
:10DFA000704000F0D3BEA572E6727CBD582D020011
:10DFB0004820002073645F626C655F6761747463FE
:10DFC0005F65786368616E67655F6D74755F7265C4
:10DFD000717565737428292072657475726E656435
:10DFE0002025732E0000000020B10278DE2A03D025
:10DFF000082070470E20704741800020704760B1B4
:10E0000059B10278DE2A0AD009684160DE21017028
:10E010004FF6FF714180002070470E2070470820A6
:10E0200070477FB5054600294DD0002D4BD00878AC
:10E030000C46DE2847D1A8886188884202D1204654
:10E0400004F070FB2888012825D002283BD0112835
:10E050003AD0512837D135F8040F6188884232D13F
:10E06000A978A81C02292ED1017A042903D00629F7
:10E0700001D0052927D10021009102228DF800202E
:10E0800001914FF4C07202910391ADF80420007A1F
:10E0900005280FD010E0297A2046012913D1A9883C
:10E0A000428891420FD10121017204B0BDE8704055
:10E0B00004F038BBADF8041028886946B0DF0028AA
:10E0C00001D0616888477FBDA88861888842FAD1FD
:10E0D0004FF6FF7060807FBD00F18040006800282F
:10E0E00000D00120704708B500F180400021016098
:10E0F0000068009008BD000070B50B4C207808B196
:10E1000085250FE00020A06060602061E060074886
:10E1100001F03AFA054601F095F908B901F01EFA46
:10E1200001202070284670BDF428002095B701001A
:10E1300038B500258DF800506846FBF7A5FF074C61
:10E14000E068401EE060E06810B901F02DFAA570AB
:10E150009DF80000FBF7BCFF38BD0000F42800204C
:10E1600070B5064604780C4888B0154640F824205F
:10E17000094A0869121D42F8240020226846FBF76C
:10E1800075F904940DB1054A00E000226946301D7E
:10E1900001F032FB08B070BDFC1E0020812402009B
:10E1A0000FB408B50399002904D004AA00926A4666
:10E1B00000F00FF801B05DF814FB10B5826804465A
:10E1C000002A05D0D4E90403216898470020A06004
:10E1D00010BD2DE9FC4791460C00804676D014F81E
:10E1E000011B39B125290ED04046FDF729FA2078C8
:10E1F0000028F4D198F80C00002867D04046BDE80C
:10E20000FC47FFF7DABF0020012221782B291BD021
:10E210002D2902D0302908D102E040F0010001E0B0
:10E2200040F00200641C002AEFD100252A290ED0FC
:10E230002178A1F130020A2A11D205EB850201EB07
:10E240004205641C303DF1E740F00400EAE7D9F8EC
:10E2500000100B1DC9F800300968641C0D442178BA
:10E2600000232E290BD114F8011FA1F130020A2A34
:10E2700005D203EB830201EB4203303BF3E76C2949
:10E280000DD068290BD0692921D00BDC252918D0A5
:10E29000582931D063290ED0642915D117E014F81C
:10E2A000011FECE7702969D0732932D075291BD082
:10E2B000782909D120E0D9F80000011DC9F8001023
:10E2C00001784046FDF7BCF9641C90E76CE0D9F892
:10E2D00000100A1DC9F800200968CDE900500A2283
:10E2E0004046FEF789FFEFE7D9F800100A1DC9F88C
:10E2F000002009680A2206E0D9F800100A1DC9F8B2
:10E30000002009681022CDE90050404604F060F971
:10E31000DAE7D9F8001000270A1DC9F800200E68B6
:10E32000C00705D112E04046761C7F1CFDF788F936
:10E3300031780029F7D104E0202140466D1EFDF719
:10E340007FF9BD42C0D9002DF6D1BDE74EB13046B0
:10E35000FBF7B0F8074604E0202140466D1EFDF7AC
:10E360006FF9BD4206D9002DF6D103E04046761C78
:10E37000FDF766F931780029F8D1A5E7D9F8000052
:10E38000011DC9F80010056830214046FDF758F915
:10E3900078214046FDF754F908200021CDE900011D
:10E3A000034610222946B0E7BDE8FC872DE9F84F67
:10E3B0002B4E04009A4630884FF0010315468946DB
:10E3C00003EB004024D0216800292BD0002D32D04F
:10E3D000626849464FF010071268A2F1010C1CEA6E
:10E3E000090F11D198466A432046FBF7AFFB00287E
:10E3F0002AD0206853462A46066901B0494620467D
:10E40000B446BDE8F04F6047164B17A2009721E0D5
:10E410000E210091134B1EA21FA100F0A6FC0E209E
:10E42000BDE8F88F082100910E4B26A21AA100F03A
:10E430009CFC0820F4E7092100910A4B24A216A1B4
:10E4400000F093FC0920EBE700973188054B214A47
:10E4500008EB014010A100F088FC1020E0E700006C
:10E46000682000207F2E0200616464725F69735F20
:10E47000706167655F616C69676E656428705F666F
:10E48000732C20706167655F61646472290000000D
:10E49000705F667300000000257320636865636B1E
:10E4A000206661696C656420696E202573282920C7
:10E4B000776974682076616C756520307825782ED0
:10E4C00000000000705F66732D3E705F6170690030
:10E4D0006C656E003432020038B503000F484FF00F
:10E4E00001054FF00E04008805EB004009D061B132
:10E4F00019600C6801B0A446BDE8304011461846CA
:10E500006047074B07A2009402E0054B07A2009466
:10E5100008A100F02AFC0E2038BD00006820002071
:10E52000342E0200705F667300000000705F61703F
:10E5300069000000257320636865636B206661696C
:10E540006C656420696E20257328292077697468BA
:10E550002076616C756520307825782E00000000EB
:10E560002DE9F04128B1016819B1C969BDE8F04150
:10E5700008470D4D0D480024461B14270DE000BF31
:10E5800004EB840005EB8000016829B1C969884764
:10E5900010B10120BDE8F081641CB6FBF7F0A04289
:10E5A000EED80020F6E700003020002044200020B4
:10E5B000044801214174007A08B10020704701200D
:10E5C000704700002C2C0020012801D0032808D11E
:10E5D0000449002201284A7400D00020087402F087
:10E5E00027BF70472C2C002070B50246022801D0AE
:10E5F000032A45D1234C207A002841D0012833D06A
:10E60000022831D120480023022A006802D0032AC0
:10E610002AD11BE0E360017911B1012924D10DE079
:10E62000D0E90565711B4FF48056B14200D33146E5
:10E63000294481614569A9420ED015E00169491C50
:10E640000161426991420FD1237213E0E168491CD4
:10E65000E160082908D9E3602372022A0AD00D215B
:10E66000FDF7A4FD02F08AFE607C28B1BDE8704091
:10E6700000F0EEBE0021F3E7BDE8704002F0D8BE26
:10E6800070BD00002C2C0020AC1F00202DE9F84F9D
:10E690003A4D04008B4628884FF00106DDF828A08B
:10E6A000984691464FF00E0106EB00401AD0B9F1A2
:10E6B000000F1BD02168002920D00921B8F1000FDC
:10E6C00025D062685368B8FBF3F703FB1782002A72
:10E6D00021D02B4B2BA2009135A100F046FB092045
:10E6E000BDE8F88F264B3DA2009102E0244B3DA2ED
:10E6F00000912FA100F039FB0E20F1E708210091D5
:10E700001F4B3AA22AA100F030FB0820E8E71C4B7F
:10E7100039A20091E0E75846FBF712FA102798B1AA
:10E720004846FBF70DFAB0B1424659462046FBF782
:10E730000DFAB8B1CDF800A0206843464A46C56836
:10E7400059462046A847CBE7009728880C4B06EB94
:10E7500000402AA20CE000972888094B06EB0040F5
:10E760002CA205E000972888054B06EB004032A25A
:10E770000FA100F0FAFA1020B2E700006820002094
:10E780006C2E020021286C656E202520705F667358
:10E790002D3E705F666C6173685F696E666F2D3EBB
:10E7A00070726F6772616D5F756E69742900000029
:10E7B000257320636865636B206661696C656420FE
:10E7C000696E202573282920776974682076616C2A
:10E7D000756520307825782E00000000705F667324
:10E7E00000000000705F737263000000705F66736A
:10E7F0002D3E705F617069006C656E0061646472CB
:10E800005F69735F616C69676E6564333228646544
:10E8100073742900616464725F69735F616C696716
:10E820006E65643332282875696E7433325F7429DB
:10E83000705F737263290000616464725F69735F63
:10E8400077697468696E5F626F756E647328705F54
:10E8500066732C20646573742C206C656E2900002F
:10E8600070B541EA4201DDE904564FF0A04441EAA7
:10E87000830141EA052104EB800041EA0641C0F82A
:10E88000001770BD70B541EA4201DDE904564FF052
:10E89000A04441EA830141EA052104EB800041EAFA
:10E8A0000641C0F8001770BD70B541EA4201DDE9CC
:10E8B00004564FF0A04441EA830141EA052104EBEC
:10E8C000800041EA0641C0F8001770BD1CB5002168
:10E8D00000910B4601220191FFF7E6FF1CBD1CB51C
:10E8E00000220B46009211460192FFF7DDFF1CBD8E
:10E8F0001CB5002100910B46012201911146FFF742
:10E90000D3FF1CBD4FF0A04202EB8000D0F80027DF
:10E9100022F44032C0F80027D0F8002742EA014133
:10E92000C0F80017704701224FF0A043824011B198
:10E93000C3F808257047C3F80C25704718B5084B75
:10E940006C4601441B68009306E000BF54F8203079
:10E95000D3F81035401C08C28142F7D818BD00001A
:10E96000F42D0200034908B5084400210160006845
:10E97000009008BD0060004002494058012800D0C6
:10E98000002070470060004030B5124B0146002067
:10E99000D3F81044224609E0157A854205D1401C7F
:10E9A0000A28F7DB4FF0FF3030BD5268002AF3D160
:10E9B000421CF9D00872D3F810242AB152684A6078
:10E9C000D3F81024516030BD0022C3F810144A60FF
:10E9D00030BD00004C2D0020F0B595B01C4615460A
:10E9E0000F4608461A9E00F01BFB182109A8FAF7EB
:10E9F00056FD0E96CDE909540023082203A9384696
:10EA000000F023FB05980690BDF81000ADF81C003F
:10EA1000BDF81200ADF81E0000208DF8210003980B
:10EA2000082600F00300012802D0022818D032E0A6
:10EA300003983346850AC0F3C2008DF8200003987E
:10EA40000FA9C0F38314A200384600F0FEFA09A80B
:10EA5000009006AB22460FA9284600F03DFA1AE0C6
:10EA60000398840DC0F3C2008DF82000082C01D259
:10EA7000254600E0082533462A460FA9384600F00F
:10EA8000E4FA2E44641B09AB06AA29460FA800F03D
:10EA900075F9002CEAD1384600F0C8FA15B0F0BD7F
:10EAA0007047012003F0C4BC10B5044800F030FFEB
:10EAB000BDE81040002003F0BBBC0000C41F0020D4
:10EAC00008B5034A00924023024AFFF785FF08BDBC
:10EAD000F51B02004C2C00200A4A012902EBC00061
:10EAE00007D0022907D0032907D0042907D0002026
:10EAF00070470220704704207047007970474079C2
:10EB0000704700004039020010B5FFF7CAFF04212A
:10EB10000348FFF739FF02490120487210BD000089
:10EB2000CC1F00202DE9F04F8DB0FCF799FD18B1F6
:10EB300000200DB0BDE8F08F7A4C4FF0000BC4F808
:10EB400018B4BFF34F8F60680290A568D84628407C
:10EB500004EB800008E021680298814201D86160DE
:10EB6000E6E7284004EB80000C3002A9FEF7D8FB52
:10EB70000028F0D105AA029901EA050304EB8303FA
:10EB8000491CDB6842F82030401C02910228F2D375
:10EB9000059800F00300022802D001284ED0A9E019
:10EBA00005985022810D8946B2EB905F00D8502124
:10EBB0000E4666F39F50059008315B4800F0E7F978
:10EBC000070079D000F02CFA4346082205A9384600
:10EBD00000F041FA029908F1080A2940681A8000F9
:10EBE000001D864223D94F4D0C3530B1C2B204EB23
:10EBF0008101301A90460C3104E02946F2B200251A
:10EC000090462846C6B25346384600F024FA0AEB2E
:10EC100008032DB1324629464FEA070000F01BFADF
:10EC2000029909F1030001EB900002903BE004EB34
:10EC300081015346324638460C31EFE70598C0F360
:10EC40008310062800D30620059960F38911C1F3CB
:10EC50008310801C05918100334800F098F907006B
:10EC600048D000F0DDF94346082205A9384600F0F7
:10EC7000F2F908F1080800260FE00298434600EA7E
:10EC80000501401C04EB81010290042238460C313E
:10EC900000F0E1F908F10408761C0598C0F3831030
:10ECA000B042EAD847B1D4F81054D4F8180468B187
:10ECB000384600F0BBF92FE01CE0687A012804D147
:10ECC0002A6828463946126890476D68002DF4D1AD
:10ECD000384600F0ABF98DF800B06846FBF7D4F980
:10ECE000D4F8180408B9029860609DF80000FBF79A
:10ECF000EFF911E0D4F8104404E021682046896857
:10ED000088476468002CF8D108480221008801EB8C
:10ED1000004007A100F016F8FCF7A2FC80F001000B
:10ED200007E700004C2D0020C839020078200020A1
:10ED30004261636B656E647320666C7573686564AD
:10ED40000000000000231A4603F024BA08B501238E
:10ED500000926A4603F01EFA08BD1CB5CDE90023F7
:10ED600002236A4603F016FA1CBD3EB5069C8DE8E8
:10ED70001C0003236A4603F00DFA3EBD2DE9F0475F
:10ED80000E4680461C46924608293ED894F80C90C0
:10ED9000002020731946104602F08EFA0025B54275
:10EDA00006D218F805201AA12046FFF7F9F903E06A
:10EDB00019A12046FFF7F4F96D1C082DEFD317A118
:10EDC0002046FFF7EDF90025B54210D218F805707E
:10EDD000FAF748FB0068C05D10F03E0F01D03A46DC
:10EDE00000E02E220EA12046FFF7DAF903E00DA184
:10EDF0002046FFF7D5F96D1C082DE5D301222146E9
:10EE0000504602F03BFA84F80C90BDE8F087000011
:10EE10002025303278000000202020007C000000F7
:10EE20002563000020000000104810B5FF2181601C
:10EE3000002101604160C0F81814C0F8141480F873
:10EE400020140B4800F0F0F800280DD109480A49B9
:10EE50000A4B401AC108002003E000BF23F820003D
:10EE6000401C8842FAD3002010BD00004C2D002029
:10EE7000C8390200C839020040390200442000208D
:10EE800002480349401AC00870470000C839020010
:10EE90004039020013B56846FEF736FE08B100207F
:10EEA0001CBD0248009950F831001CBD40390200D9
:10EEB00070B508480125D0F8104480F8205405E0CA
:10EEC000657221682046496888476468002CF7D13C
:10EED00070BD00004C2D00202DE9FF4781460C9DA0
:10EEE00000200C462F7B2873984616462946184664
:10EEF00002F0E2F9072E42D2DFE806F004090F160D
:10EF00001F2A360049462846FFF74AF937E04946A6
:10EF100028462268FFF744F931E0D4E90023494646
:10EF20002846FFF73DF92AE0A0680090D4E90023C5
:10EF300049462846FFF734F921E0D4E90201CDE93A
:10EF40000001D4E9002349462846FFF729F916E0D5
:10EF500004F1080007C88DE80700D4E900234946FA
:10EF60002846FFF71DF90AE004F108000FC88DE8F4
:10EF70000F00D4E9002349462846FFF711F9002283
:10EF80002946404602F07AF92F73BDE8FF872DE944
:10EF9000F041858A80462D1F4819C01CB0FBF5F052
:10EFA000C6B24046FEF735FF041E19D0002020717E
:10EFB00001206071E58000272546761EC4F8008098
:10EFC0000BE04046FEF725FF60B16179491C617195
:10EFD000286005467F1CC0F80080B742F1D3204668
:10EFE000BDE8F081204600F002F80020F8E72DE9A6
:10EFF000F041457901466B1E002201E00968521C70
:10F000009A42FBD30F680146002605E038460C689B
:10F01000FEF721FF2146761CAE42F7D3BDE8F08112
:10F020000121001DFEF7C9BEFEF72DBF10B5044635
:10F030000121001DFEF7E7FE10F0FF0F04D120466E
:10F04000BDE81040FFF7D3BF10BD38B501240094D0
:10F05000FEF71EFD38BD38B500240094FEF718FDFC
:10F0600038BD0000064910B500204870091D086031
:10F07000BFF35F8F0349044800F016FA002010BD6B
:10F08000B41F0020DC2E0200402C002010B500F040
:10F09000D9F908B141DF10BD20BF40BF20BF10BD6E
:10F0A000FAF7D0BE20B1034909680160002070471B
:10F0B0000E207047C8300200FEB502460E460846D4
:10F0C000FFF7F0FF002868D1002400940194012587
:10F0D00006208DF80020ADF8040002948DF802504F
:10F0E00069462020326869DF2C4F48B100F020FAD1
:10F0F0003988024605EB014329491846FFF726FEE9
:10F100000094019402948DF80150694640203268C1
:10F1100069DF40B100F00CFA02463888214905EB5E
:10F120000040FFF713FE0094019402948DF8004014
:10F1300069460120326869DF40B100F0F9F9024602
:10F140003888194905EB0040FFF700FE4FF4B06026
:10F150000090019402946946A120326869DF40B1B1
:10F1600000F0E6F902463888104905EB0040FFF749
:10F17000EDFD0094019402948DF800406946A020B2
:10F18000326869DF40B100F0D3F902463888084997
:10F1900005EB0040FFF7DAFD0020FEBD80200020D7
:10F1A000CC370200143802002C37020078370200F6
:10F1B000D83602002DE9F0410446D0F8008060DF27
:10F1C0002168194D074641451CD92888022606EBBF
:10F1D000004016A1FFF7B6FD2888424606EB004026
:10F1E0001EA12368FFF7B9FDF006D0F80C012168D5
:10F1F000800200F10050421A288825A106EB004049
:10F20000FFF7A4FD012467B1384600F091F90246EA
:10F2100028882AA104EB0040FFF798FD3846BDE896
:10F22000F0812E480470F9E780200020496E737544
:10F230006666696369656E742052414D20616C6C2D
:10F240006F636174656420666F7220746865205313
:10F250006F66744465766963652E00004368616E6D
:10F260006765207468652052414D20737461727423
:10F27000206C6F636174696F6E2066726F6D2030F1
:10F2800078257820746F20307825782E00000000D3
:10F290004D6178696D756D2052414D2073697A65B5
:10F2A00020666F72206170706C69636174696F6E43
:10F2B00020697320307825782E00000073645F6227
:10F2C0006C655F656E61626C652829207265747576
:10F2D000726E65642025732E000000002B20002034
:10F2E00030B5144891B00078002820D05FF0340584
:10F2F000ADF8405010A903A861DF30B1052816D041
:10F3000011B0BDE83040FAF79DBD03AC0A4968462C
:10F3100000F0CAF807E000BFD0E90021204690477E
:10F32000684600F0D8F802980028E1D0F4E711B060
:10F3300030BD00002B200020CC300200F8B5134C6B
:10F340002078C0B10120A07002F0B4FA112814D0C6
:10F35000022002F0C7FA00258DF800506846FAF73F
:10F3600093FE11DF064625709DF80000FAF7B0FE07
:10F370002EB13046F8BD0820F8BD0020F8BDA570BC
:10F3800002F0C4FE032002F0ADFAF6E728200020C8
:10F390007CB5204C207808B108207CBD0120A070ED
:10F3A000002002F087FA112819D0002002F09AFA02
:10F3B00019480026006801908DF800606846FAF749
:10F3C00063FE164901A810DF05000AD00020207056
:10F3D0009DF80000FAF77CFE2DB128467CBD002088
:10F3E0007CBD0120F3E7A67066700721162002F0AD
:10F3F00017FA08B1FAF726FD0721152002F010FAD6
:10F4000008B1FAF71FFD02F09DFE012002F06AFA32
:10F41000E5E700002820002060300200C99D0100BF
:10F420000EB50749684600F03FF805E0D0E9001046
:10F430008847684600F04FF802980028F6D10EBDC4
:10F440007C3002000148007870470000282000202E
:10F450000548817819B1007818B1FFF76FBF08200F
:10F460007047FFF795BF0000282000201FB56846B1
:10F470004BDF30B1052814D004B0BDE81040FAF7D6
:10F48000E1BC084901A800F00FF806E0D0E900212E
:10F490000098904701A800F01EF803980028E6D0D5
:10F4A000F4E71FBDE8300200016009684160AFF376
:10F4B000008010B5D0E900215368994201D10021A4
:10F4C00004E0D1E90034A34202D01946816010BDA6
:10F4D00008314160F0E7816800290BD0026892682A
:10F4E0000A44826041684B689A4203D10831416006
:10F4F000FFF7DFBF704700000C4A10B502F59473A8
:10F500000EE0991AC91001EBD171491002EBC1014B
:10F510000C68844201D90B4602E005D201F10802D1
:10F520009A42EED3002010BD486810BDFC2E0200A8
:10F5300000B5FFF7E1FF002800D1014800BD000041
:10F54000E82E02004058002800D00120704708B57E
:10F55000002242504058009008BD00000848006852
:10F56000012110F0010F08D14FF0E020E02280F8D7
:10F570000024C0F88012C0F80011024801607047F2
:10F5800000E100E0180500400649024600200B7922
:10F590000BB1852070470A6001220A7100224A716E
:10F5A00070470000041F002004490120086004483F
:10F5B0000168C1F300410029FAD170470C000040F6
:10F5C00018040040002802D0014980010847704714
:10F5D000052E02002DE9F0418846054601F066FA45
:10F5E000234E002828461AD0FCF77AF8304490F8C9
:10F5F00048008009032802D001280ED007E04FF010
:10F60000A040D0F81005E84010F0010F05D003210C
:10F610002846BDE8F041FFF775B90221F8E701F08F
:10F6200051FA002822D02846FCF75AF804464FF435
:10F63000807000EB84000F4F81B207EB8400D0F89C
:10F64000102542F00102C0F810250846FFF78AF99C
:10F65000B8F1000F0AD02846FCF742F856F820000F
:10F66000002803D00120A040C7F80403BDE8F081C2
:10F6700008290020006000402DE9FC41DFF8BC8033
:10F68000044608EB0400002790F930001346C01729
:10F690000E46401C01D008274CE0B0781946C0F354
:10F6A00040022046FBF7F8FF0546401C41D0B078E9
:10F6B000410719D4C0070AD04FF0A04000EB8401E5
:10F6C000D1F8000720F00200C1F8000707E0002190
:10F6D0007378204600910A460191FFF7D3F8174945
:10F6E00020465431FEF7EFFBB078800718D5144858
:10F6F000317800EB8500D0F81025124B1A40C0F885
:10F7000010254FF4F8524FF4403302EA042203EA82
:10F7100001410A43D0F810150A43C0F8102509E04A
:10F7200008EB0500327810F8481F41EA8211017099
:10F7300000E004273846BDE8FC81000008290020CD
:10F7400000600040FFE0FCFF4FF0A041D1F8101531
:10F75000C14011F0010000D00120704770B5184D74
:10F7600095F8580008B1082070BD0020411E2A18E5
:10F77000401CC0B282F830102028F8D30024204664
:10F78000FBF77CFF641CE4B20C2CF8D300240D4979
:10F79000E0206C6581F8000401264020891FC1F833
:10F7A0008002C1F800014FF4BE70FFF7DBF8064994
:10F7B000F007C1F8040385F85860204670BD0000CA
:10F7C0000829002006E000E000600040034890F8AF
:10F7D0005800002800D001207047000008290020B0
:10F7E0000121B1EB507F01D101207047002070470B
:10F7F00000207047704700002DE9F041054616468D
:10F8000000790F46154A00EBC00102EB810494F821
:10F81000201011B10820BDE8F081114951F82010E5
:10F820002868FFF7E5FF08B11120F4E739462846BC
:10F83000FAF768FC6660386920601EB1397F284697
:10F84000FDF72EFD28680821C0F800150020A061F2
:10F85000E0610121606184F82010DCE76429002068
:10F86000F82D02002DE9F04704460E4600792049A4
:10F8700000EBC00001EB800517463046FFF7B0FFF4
:10F8800030B1204600F036F820B11120BDE8F087F5
:10F890001020FBE76F61AE604FF490760027314691
:10F8A0002068FFF754FE4FF4AC7841462068FFF71C
:10F8B0004EFE2068AA686969C0F84425C0F848155A
:10F8C000206801218160686878B9B146494620689E
:10F8D000FFF738FE064641462068FFF733FE064331
:10F8E000F4D000B10F27002068613846CEE7000051
:10F8F000642900200079054900EBC00001EB80007D
:10F900004069002800D001207047000064290020D1
:10F910002DE9F04704460079274900EBC00001EBD0
:10F92000800720684FF00009C0F80095786880B122
:10F9300020682249C0F8081320680121000B40B25A
:10F9400000F01F0291404009800000F1E020C0F863
:10F9500080112068D0F80C25D0F81485D0F80865FF
:10F96000D0F810554FF0FF31C0F80C15C0F8141541
:10F970002068C0F80815C0F81015501C02D01046B9
:10F98000FEF7A4FFB8F1FF3F02D04046FEF79EFF0E
:10F99000681C02D02846FEF799FF701C02D0304642
:10F9A000FEF794FF2068FFF725FF87F82090C7F83F
:10F9B0000490BDE8F08700006429002010030200D5
:10F9C00000B52A490322B1B00988082802EB014298
:10F9D0004AD2DFE800F02C4949040A181E311046CB
:10F9E00023A1FFF7AFF9022004E0104625A1FFF79D
:10F9F000A9F90420FBF7A6FC002835D031B05DF84A
:10FA000004EBFAF71FBA104623A1FFF79BF9032076
:10FA1000F0E7104628A1FFF795F90320FBF792FCC9
:10FA200008B1FAF70FFA2C48FAF7D4FDE4E731B041
:10FA30005DF804EB02F038B908202F90309030AB1D
:10FA400001AA2FA921A801F0F9FB08B1FAF7FAF9E8
:10FA50003098009001AB21A91F482F9AFAF7DFFEDA
:10FA6000002801D0FAF7EEF931B000BD782000206F
:10FA700046617374206164766572746973696E6738
:10FA800000000000536C6F772061647665727469C2
:10FA900073696E67000000004661737420616476CC
:10FAA0006572746973696E67207769746820576836
:10FAB0006974654C69737400536C6F772061647668
:10FAC0006572746973696E67207769746820576816
:10FAD0006974654C69737400842100202DE9F84F26
:10FAE00005460C460888B5F8CA12884259D195F8DF
:10FAF000C602DFF8F8A000EB8001C1EB801005EB37
:10FB0000400160884FF003094FF00008F0BBE68821
:10FB10000879A21DF3B250FA86F6062E01D80344E6
:10FB200000E006230B7100261CE000BF00EBC003C1
:10FB300006EB860702EB470701EB4303D7F802C049
:10FB4000C3F80AC0D7F806C0C3F80EC07F895F8229
:10FB5000A3F81480A3F81680A3F81880401CA3F81B
:10FB60001A80761C0B798342E0D895F8C62200EB08
:10FB7000C00002EB8203C3EB821205EB420231F8B4
:10FB80001000128990420ED2087900E00BE006289E
:10FB900009D085F8C50221882846FBF7A9FD010098
:10FBA0000AD1BDE8F88F85F8C582228869462846C3
:10FBB000FCF736F901000BD085F8C7822288284669
:10FBC000FCF708FA8AF800902188AAF80210E8E702
:10FBD0009DF800000028E4D0228801212846FCF787
:10FBE000B1F92188284600F0E1F9DAE798230020EE
:10FBF0000078002807D104483B21008876DF0028E0
:10FC000001D0FAF71FB97047481B002070B50246B3
:10FC10008888C97B00EB400302EB4304A41D012943
:10FC200001D11188218021886288914211D9A5DFF4
:10FC3000012568B111280DD0FFF77AFC024606486D
:10FC400006A1008805EB0040BDE87040FFF77EB8D4
:10FC5000657170BD257170BD4820002073645F62BE
:10FC60006C655F67617474635F65786368616E6714
:10FC7000655F6D74755F7265717565737428292091
:10FC800072657475726E65642025732E0000000025
:10FC900010B51B480C46097803220088052902EBA1
:10FCA00000402CD2DFE801F0030C1C1E260015A139
:10FCB000FFF748F86188221D1D48FAF7A1FE09E008
:10FCC0001CA1FFF73FF86088A0F57F41FF3916D0EF
:10FCD000132176DF002812D0BDE81040FAF7B2B841
:10FCE0001FA108E024A1FFF72DF82046BDE8104031
:10FCF000FBF78CBE26A1BDE81040FFF723B810BD6E
:10FD00007820002043757272656E742054696D65A9
:10FD1000205365727669636520646973636F7665E5
:10FD2000726564206F6E207365727665722E0000B6
:10FD30005821002043757272656E742054696D6598
:10FD40002053657276696365206E6F7420666F75E7
:10FD50006E64206F6E207365727665722E200000CF
:10FD6000446973636F6E6E65637420436F6D706C6E
:10FD70006574652E0000000043757272656E742014
:10FD800054696D652072656365697665642E00004F
:10FD9000496E76616C69642054696D652072656393
:10FDA00065697665642E0000F8B505460C4608883E
:10FDB000B5F8CA1288425DD195F8C602A61D00EBBF
:10FDC0008001C1EB801005EB400395F8C502618806
:10FDD00000EBC00003EB40000A3039B329E000BF5C
:10FDE00001EB410206EB42029788B7F5245F0CD085
:10FDF0006FF4245C17EB0C070AD0012F02D0072FF9
:10FE00000BD108E05288428107E05288828104E0E9
:10FE10005288C28101E05288028242892AB18289D5
:10FE20001AB1C2890AB1028A1AB9491C32888A42B7
:10FE3000D6D800268DF8006095F8C5021979401CC7
:10FE4000884203D101208DF8000018E085F8C50232
:10FE5000228869462846FBF7E3FF01000BD085F8AE
:10FE6000C76222882846FCF7B5F80A4803210170CA
:10FE700021884180F8BD9DF800000028FAD0228832
:10FE800001212846FCF75EF82188284600F08EF80C
:10FE9000F8BD0000982300207CB506468D88C888F0
:10FEA00005EB450106EB4104A41D172800D21720DD
:10FEB0002188814200D80846608000202071218876
:10FEC0002846B5DF50B1FFF733FB02460E4801214B
:10FED000008801EB00400DA1FEF738FF6079002893
:10FEE00010D1F06800280DD01449D1E90201CDE904
:10FEF0000001ADF802506088ADF80400F268694670
:10FF0000304690477CBD00004820002073645F624B
:10FF10006C655F67617474735F65786368616E6751
:10FF2000655F6D74755F7265706C792829207265E4
:10FF30007475726E65642025732E0000582D0200C2
:10FF400070B505460C4690F8C602228800EB800189
:10FF5000C1EB801005EB4001B5F8CA02824222D104
:10FF6000608848B100212846FBF7ECFF218828462D
:10FF7000BDE8704000F01AB8A2680A60E068C1F8F5
:10FF8000060021882846FBF7B3FB01000BD00020B8
:10FF900085F8C70222882846FCF71CF8024803218E
:10FFA00001702188418070BD982300202DE9F04127
:10FFB000044690F8C9020E46401C1949C0B284F8A4
:10FFC000C902C9680327174D4FF0000E884224D29A
:10FFD00084F8C5E294F8C602401CC0B200EB800170
:10FFE000C1EB801104EB410284F8C602A5F11801AF
:10FFF00001EB800001210068106082F804E03046C7
:020000040002F8
:100000009BDF010007D084F8C7E232462046FBF7A9
:10001000E1FF2F706E80BDE8F08184F8C7E2F8E759
:10002000941E00209823002048B1064A016891429E
:1000300005D140680449401802D0012800D00320AF
:1000400070470000DEC0ADDE02FEE10E8A7D022AAE
:1000500004D90289CB881A44D21C02814289C988FA
:10006000511AC91E418170472DE9F0410D46022108
:10007000904600F58056298000F10804144F1BE0DB
:1000800031462046FCF7DAFD40B1B8F1000F02D04E
:10009000012288F80020022816D004E0A0687969BF
:1000A000884200D97861288861880844C01C28806B
:1000B000608804EB80040C3431462046FCF7D1FD07
:1000C0000028DDD1BDE8F0814FF480602880F9E799
:1000D000681F002008B50021009101460823024A4C
:1000E0000248FEF7D3FA08BD1C2E02003020002083
:1000F00008B50020009004480823044A0168044819
:10010000FEF7C4FA08BD0000901F0020142E020064
:10011000302000202DE9F05F0025DFF80891DFF89E
:1001200008B12C464FF00308AA462F46D9F80C0018
:1001300000EB07363046FFF777FF78B3012847D04A
:10014000032862D100204FF4806200BF56F82010CF
:10015000491C0ED004EB84010BEB8102A8F10100D5
:10016000566003221FFA80F80BF82120641CA4B209
:100170004BE0401C9042E9D32C48016879B104EB74
:10018000840102200BF821000BEB81014E600881F5
:10019000254828304480641CA4B205E007E0022111
:1001A000066081804FF0010A45F001052DE004EB67
:1001B000840100220BF821200BEB810101F11002D8
:1001C0004E6030460831FFF74FFF45F00205CDE79E
:1001D000BAF1000F0CD0022004EB8401134A0BF893
:1001E00021000BEB810112684A60641C0881A4B2F3
:1001F0000E480022011D06603046FFF735FF0B4810
:10020000808802280CD0082005437F1CBFB2032F32
:100210008CD3B8F1020F00D20025E8B2BDE8F09F00
:100220000420F1E730200020682B0020901F0020E0
:1002300001494978FAF796BBD81E0020002101F049
:1002400039BF30B585B00C4605218DF80010154634
:10025000ADF80200FCF7C4FEADF804006846CDE935
:100260000245FCF739F805B030BD000070B5054D0A
:1002700006460024304655F824108847641C032C99
:10028000F8D370BD802D02003EB5104D002400BF94
:1002900005EB041002F0A0FB641C022CF8D301242F
:1002A000502002210094CDE901100849084BB039D3
:1002B000A02201F1A00000F03FFC08B103203EBDE8
:1002C0000348401E847000203EBD000048280020E6
:1002D000C51E002000F06CB900F06CB970B5044682
:1002E0000025C168184A284602EB00139B688B4220
:1002F00002D102EB001003E0401C0228F4DB0020D6
:100300002178082904D0092908D0132914D112E032
:10031000617A89B980B102F06FFB0DE0617A59B959
:1003200050B100218160817B41F002018173074956
:100330000120087003E001252046FFF797FF2846BB
:10034000BDE8704001F000B948280020C41E00201C
:1003500000F0E5B908B513889B0000936B4600F0E8
:100360005FF908BD002300F05BB938B505460024ED
:10037000204609E08178284600F080F810B1052871
:1003800000D003240098401C00906946284602F0E3
:100390000FFB0028EED134B9284600F0C4F910B1A3
:1003A000072802D00324204638BD0724FBE7134664
:1003B000002200F069B900002DE9F0471F00154642
:1003C0000E46814604D0072E05D0082E16D102E035
:1003D0000E20BDE8F0878DB1022D0FD800F0AEF9E8
:1003E00060B14FF000083146484602F0C7FA041EDB
:1003F00006D0207BA8420DD00F20EAE70720E8E7CF
:10040000FF214FF6FF7002F0B9FA041E06D0A0F8E3
:100410000090A670607BFF2802D00CE01120D8E786
:100420002946154800F05AFB014620466173FF2912
:1004300013D04FF001082573617B0F4800F09CFB3F
:1004400002000DD0ABB23146384600F007FAB8F1E1
:10045000000F0ED0082E05D00BE002F0BDFADDE74C
:100460000320B6E738886FF0050101EB800079685A
:1004700088800020ADE700003828002070B50024F7
:1004800002F07CFA05000BD0686820B100F06FF92B
:10049000040000D00324284602F0AEFA204670BDC6
:1004A000052070BD70B515460C46072903D0082CF1
:1004B00001D0072070BD02F061FA28B10580847078
:1004C000BDE8704002F018BA052070BD7CB50D463D
:1004D000072903D0082D01D007207CBD002602F09B
:1004E0004DFA040002D0606810B11CE005207CBD0C
:1004F000617B0F4800F040FB02004FF000000090CD
:1005000001908DF8025010D0237B2946684600F0F8
:100510003DF9684602F0DEF9211D684600F010F949
:100520000646092801D030467CBD03207CBD000072
:10053000382800204FF6FF714180014909680847BB
:10054000682D020030B587B01748FCF74FF810B19E
:10055000032007B030BDFBF76BFF08B18620F8E73A
:1005600000F0CEF9002002904CF2070403900EE058
:10057000694604A8FCF704F800988088A0F540407C
:1005800085B204A8FBF7BCFF284600F075F902AA63
:1005900004A92046FBF7DBFF0028E9D0034901202E
:1005A00008700020D5E70000E5C20100B81E002059
:1005B00000F088B900F08CB970B586B014460E46CC
:1005C000054600F03BF940B105F5404080B20F4AC6
:1005D0006946FBF7BCFF40B902E0012006B070BDE0
:1005E00003A96846FBF7CCFF08B10020F6E7A57029
:1005F0000398408820800498606003988088A0F564
:10060000404030806846FBF77BFFE6E7BC1E0020D9
:10061000024800214160816070470000B81E002040
:10062000F0B587B01D46144607460E46FF280AD887
:10063000084600F003F930B103AA3146384600F00D
:10064000E5F840B902E0072007B0F0BD01A903A812
:10065000FBF796FF08B10520F6E7A67001984088E1
:10066000208045B18200286890420BD302996068CF
:10067000F8F7FCFE01E00298606003A8FBF740FF7A
:100680000020E1E70420DFE77FB586B01E460D4677
:100690000446FF282AD8A87800F0D0F830B304F533
:1006A0004040ADF80000A87803AA00F54040ADF83E
:1006B00002006868019028880290A978204600F01E
:1006C000A5F80528089813D010B108A8FBF7BCFFBF
:1006D000694603A8FBF778FFB0B107281DD00828AA
:1006E00019D00E2817D003200AB070BD0720FBE7F1
:1006F00028B108AA694603A8FBF771FFECE7694631
:1007000003A8FBF768FFE7E71EB1314603A8FBF734
:100710002EFF0020E8E71120E6E78620E4E74FF609
:10072000FF7000F0A9B810B5FF2801D9072010BD4F
:1007300000F0A8F800F02EF8002010BD00F0F4B88A
:1007400070B504460D46807800F078F858B12188DD
:100750002846FBF761FF002804D0072805D00928A8
:1007600000D0032070BD072070BD862070BD01B58C
:100770006846FBF769FF002800D0032008BD000091
:100780000149C978FAF7EEB8D81E00209BB200F0F4
:1007900065B8000070B51B4D8AB0002068700090ED
:1007A0004FF6FF760190304603E0204600F07CF8DB
:1007B000204600F087F80446B0421DD004F54040C2
:1007C00080B26A4602A9FBF7CAFE0A28EDD004F5FA
:1007D000404080B2FBF7ECFD08280FD000280BD07A
:1007E00005461422084905A8F8F740FEADF8184060
:1007F00005A80795FFF79EFE0AB070BD012068703E
:10080000FAE70000B81E00206C2D02007CB50546FA
:1008100016460C46084600F011F80020009005F539
:100820004045019004F54044A8B2A1B26B4632465F
:10083000FBF786FE002800D005207CBD07280BD0E2
:10084000012809D0082807D0052805D0062803D09C
:10085000042801D0002070470120704710B503EB39
:1008600083034FF6FF7404EA03138170DB1C9908BD
:100870004260018010BD00000149FAF75ABF000034
:100880006828002010B50446A0F57F40FF3807D047
:1008900004492046FAF74DFFA04201D1012010BDC6
:1008A000002010BD8828002010B50446044900F03F
:1008B00083FF03492046BDE81040203100F07CBF93
:1008C000682800200149FDF7BBB9000088280020F6
:1008D00070B50A49FDF7B4F904464FF6FF7507E015
:1008E00000F02CF838B105492046FDF7A9F9044677
:1008F000AC42F5D170BD204670BD000068280020D4
:1009000010B508484021F8F7CAFD4FF4807421461D
:10091000044800F08BFA21460248BDE81040203020
:1009200000F084BA68280020FF2803D80146024856
:1009300000F0ABBA0020704768280020FF2803D8D9
:100940000146024800F0A1BA002070478828002024
:1009500010B50C46FCF77CF8FF2804D0024900EBE8
:10096000400021F8204010BD982600201CB500F062
:1009700037FA08B1F9F766FA0020009001909DF867
:10098000000020F07E0040F00100303020F08000B8
:100990008DF8000007208DF8010010208DF802006E
:1009A0009DF8030040F003008DF803009DF804005B
:1009B00040F003008DF80400684600F02FFC08B1F9
:1009C000F9F740FA034800F013FC002801D0F9F7CA
:1009D00039FA1CBD810C02002DE9FF4F97B04FF092
:1009E0005000259E4FF0000816901D465FEA020B4E
:1009F00089464746404603D015B14FF001082860AC
:100A0000249911B10EB101273060EA461490CDF857
:100A100054D000243CE050216846F8F740FD179878
:100A200016AB14AA30F814000721FFF7F9FD0528CA
:100A30000CD007280AD09DF81100400808D00128E2
:100A400006D043F202201BB0BDE8F08F0520FAE784
:100A5000B8F1000F0FD0C4EBC40101EB0B00DDF8BF
:100A600011100160BDF8151081809DF8171081717B
:100A70002868401C286057B12498102200EB04100D
:100A80000AF10101F8F7F2FC3068401C3060641C88
:100A90004C45C0D30020D6E70068012803D00228C7
:100AA00001D000207047012070470000044908442D
:100AB00090F93000082801DB0120704700207047C2
:100AC000082900200449084490F93000082801D280
:100AD0000120704700207047082900202DE9F041CF
:100AE0000F46060026D0306820B3706810B3FF248C
:100AF00000251CE02946706800F09FF948B1FF2CE2
:100B000000D12C46281B401CB8420ED12046BDE81F
:100B1000F081FF2C06D108E02146304600F040F875
:100B2000641CE4B2AC42F7D3FF246D1CEDB2B06894
:100B3000A842DFD8FF20EAE72DE9F0410400DDE913
:100B40000705069E16D0A9B1A3B100FB05F7974291
:100B500010D8C21DB6EBD20F0CD358B155B1E56019
:100B60002160C4E9013081B2184600F05FF900202D
:100B7000BDE8F0810720FBE770B504000D460DD0FD
:100B8000206858B1606848B1FF2D07D000F07DF9AA
:100B900020B1E168206805FB010070BD002070BD38
:100BA00070B504000D4611D0206800280ED0606892
:100BB00000280BD0FF2D09D000F067F9002805D0E0
:100BC00029466068BDE8704000F06BB970BD00292F
:100BD00001D001F08DB8704770B505461B480C4632
:100BE0000078A8B1B4B12846F9F79EFEA0B102285A
:100BF000207814D020F0010020702846FCF7F0F98E
:100C0000A0F57F412078FF390CD040F008000BE0C0
:100C1000082070BD0E2070BD43F2020070BD40F090
:100C20000100E9E720F0080020702846F9F73EFEB1
:100C3000217860F3410121702846F9F75DFE2178A3
:100C400060F382012170002070BD0000C81E0020EA
:100C5000054A10B512782AB101F072F8082800D1BF
:100C6000112010BD082010BDC81E0020034A1278B4
:100C70000AB1FCF7B5B8082070470000C81E002074
:100C8000F8B504460078364E0327364D0E2834D288
:100C9000DFE800F00733143334333B6345613363DB
:100CA0004063308830A107EB0040FEF74BF81FE0AF
:100CB000002822D0BDE8F840F9F7C4B86088F9F7F9
:100CC0002BFE0246207A00903088638807EB0040B4
:100CD00030A1FEF74AF8A0886880224861880C306D
:100CE000F9F7B0FF08B1F9F7ADF8207A012804D17F
:100CF000A08800F093F91128DAD1F8BD0020009007
:100D000060886946FFF763FFF8BDFBF773FB0828AF
:100D1000FAD0CDE7BDE8F8400020F8F779BF207C95
:100D2000C007F1D0207A0728EED1A9680829EBD2B4
:100D3000284A688822F81100491C1046A960FFF76C
:100D400095FF062802D008B1F9F77CF82148A96878
:100D500000F08AFAACE72069AAE7A068A8E70000DB
:100D600078200020481B0020436F6E6E6563746519
:100D70006420746F20612070726576696F75736C82
:100D80007920626F6E646564206465766963652EA0
:100D900000000000436F6E6E656374696F6E2073B0
:100DA0006563757265643A20726F6C653A202564DC
:100DB0002C20636F6E6E5F68616E646C653A2030E4
:100DC0007825782C2070726F6365647572653A209F
:100DD00025642E003C220020FBF75ABAFBF758BAD4
:100DE00010B5FFF7AFFB88B9FFF74EFA70B900F006
:100DF00081FF58B901F0A2F840B9FBF7DFFD28B92F
:100E0000FBF79CFE10B9FCF75BF808B1032010BD9E
:100E100005484FF6FF7181800021816041700121FA
:100E20000170002010BD0000C81E0020002803D063
:100E3000C91DC908F8F733BB7047002809D001F075
:100E4000070301229A40D2B200EBD1001146FCF711
:100E500087BC70472DE9F0410D46060013D00024F1
:100E600001270EE004F0070007FA00F0C1B206EB1C
:100E7000D400FCF775FC10B12046BDE8F081641C7D
:100E8000A4B2AC42EED32846F7E740B100EBD10064
:100E900001F00702007801219140084000D00120B4
:100EA0007047F8B50400C1F3C70501F007014FF022
:100EB000010000FA01F0C6B20FD0605D30420CD0E4
:100EC00000208DF800006846F9F7DEF8605DB04359
:100ED00060559DF80000F9F7FBF8F8BD0349097863
:100EE00009B1FFF7F9B94FF6FF707047C81E00202F
:100EF0002DE9F041044686B001278088FBF75AFFB0
:100F00006080207800263F4D082808D0092820D08E
:100F10004FF6FF780A2829D00B2853D158E0607A81
:100F200010B1012809D04DE0A86830B1E1688142D4
:100F300003D1AE60A088A88016E06878E8B3A088E6
:100F4000A98888423ED1207A06283BD100F0E0FAF9
:100F500038E0607A88BBA86878B3E168814231D113
:100F6000AE60E868401EE860E6602BE0A878E8B173
:100F70004046FFF7B1F94146404517D10846FFF713
:100F8000A9F9404512D1AE7014216846F8F787FAE6
:100F90000C208DF80000ADF80480ADF80280002729
:100FA0002046FBF775F96846FBF772F9687838B1A7
:100FB000A088A988884203D100E003E000F0A8FAE5
:100FC000002F1CD006B02046BDE8F041FBF760B909
:100FD000A8780028F6D0AE7014216846F8F75FFABA
:100FE0000D208DF80000ADF80480ADF80280A068F7
:100FF00002902046FBF74CF96846FBF749F906B02A
:10100000BDE8F081C81E00200349097809B1FBF74B
:10101000D3BF082070470000C81E0020F0B52A4C3E
:10102000074687B0207838B12849D1E90201CDE9D7
:101030000501607818B104E0082007B0F0BD00F0A9
:1010400067FA6078A168401E084301D0112536E098
:10105000A088002687421CD1E068D0B10025142169
:101060006846F8F71CFA08208DF800003846FBF7B0
:10107000A1FEADF8020006208DF80800ADF804705E
:101080008DF8096003968DF810606846FBF700F94B
:1010900015E0E068411C14D0401C0B4AE0600832A7
:1010A00005A93846FFF783F9050008D0A660E06877
:1010B000401EE060112D02D0862D00D00325284669
:1010C000BBE71325FBE70000C81E00208C2D0200A3
:1010D0002DE9FF4F2A4883B09946007892468B4607
:1010E000B8B14FF6FF763046FFF7F6F8804600209D
:1010F0000090244801AA062100680190CDF808D08C
:101100004046FFF727F900256C1E3746072804D014
:1011100017E0082007B0BDE8F08F0520FAE70020AF
:101120000090A84201D305464746A04201D204469A
:1011300046464046FFF7D0F8804601AA0621FFF751
:1011400009F9D8B10528EAD0A8F57F41FF3901D0C7
:101150000320DFE70399002001B10F80BBF1000FEE
:1011600001D0CBF80050BAF1000F01D0AAF800600E
:10117000B9F1000FCED0C9F80040CBE70098D0E716
:10118000C81E00208C2D020070B5184E86B0307835
:10119000D0B10120B0704FF6FF742046FFF79CF8E5
:1011A0000546A0421DD10020B07014216846F8F712
:1011B00076F90C208DF80000ADF80440ADF802403F
:1011C0006846FBF765F80EE0082006B070BD00BF6A
:1011D000FFF71AFF08B10320F7E72846FFF77CF86E
:1011E0000546A542F4D10020EFE70000C81E00200C
:1011F000084A117821B1D178032903D3042070471C
:1012000008207047044B43F82100491CD17000208E
:1012100070470000C81E0020A82800200349097854
:1012200009B100F0BFBD082070470000C81E0020B3
:10123000002801D0FBF72CB87047000030B4094CEF
:1012400024784CB150EA020409D000B139B102B19E
:101250002BB130BCFBF7F2BE082030BC70470E202B
:10126000FBE70000C81E0020034A12780AB1FBF712
:1012700001BF082070470000C81E002010B50C46B2
:10128000017A052908D0407A38B1084808A10268D7
:101290002046FCF785FF00E01AB106A12046FCF7C6
:1012A0007FFF2046BDE81040FCF787BF04200020E8
:1012B000257300000D0A000038B5C3880D460446AA
:1012C00033B114A0009015A216A12846FCF768FFC0
:1012D000217A05291CD0607A48B1A088FDF7FCFB73
:1012E000164951F8202016A12846FCF759FFA0887E
:1012F0000021FDF7CFFD03461049207A143951F83B
:10130000202001B02846BDE830400EA1FCF748BFC0
:1013100038BD00001B5B306D000000001B5B313BE3
:1013200033316D0025734C6F67732064726F70707A
:101330006564202825642925730D0A0004200020F7
:10134000257300003C25733E2025733A20000000E1
:101350000146054810B50068FCF7A5FC04461C21B1
:10136000F8F79DF8204610BD0C2E020001460248F9
:101370000068FCF7B9BC00000C2E020003480249CB
:101380000068FCF79BBC0000B01F0020942E0200F8
:10139000F0B5254D254E85B004460027686828B96C
:1013A000214930680831FCF794FC686001460078F8
:1013B000072817D2DFE800F0160408080E0E120006
:1013C0002046FBF7ABFE02E0204601F09FFB040045
:1013D00028D008E02046FAF7E3FCF8E72046FBF7C0
:1013E000CDF9F4E70F2414216846F8F758F8A4F56E
:1013F000E8501D3800D10024019469466868FAF766
:101400008BFE6846FAF7C2FE07496F600024083178
:101410003068FCF753FC044801210C30FCF7F3FC66
:101420000028BBD105B0F0BD681F00200C2E0200C3
:101430002DE9F041234C0025234E207A012730B9B5
:101440002248311D0068FCF744FC306038B10220AE
:1014500020723168087928B101281ED116E0656034
:10146000BDE8F081D1E90503C01A4FF480529042E3
:1014700000D31046B7EB900F01D2820800E00122A2
:101480000869C9681844194429DF03E0D1E9030158
:10149000084428DF58B1112812D003213068FAF728
:1014A00085FE25726560BDE8F041FFF767BF207CCF
:1014B0000028D5D1BDE8F04100210220FDF794B805
:1014C0002772CDE72C2C0020AC1F0020942E0200A8
:1014D00010B501210448FCF77CFC002803D1BDE8CD
:1014E0001040FFF755BF10BD741F002010B5074C0A
:1014F000201DFCF75FFC002806D1607C002803D18A
:10150000BDE81040FFF794BF10BD00002C2C002058
:10151000084910B500231A46A1F10800FFF7D8FDCD
:1015200030B1052804D0002002490C39487010BDA4
:101530000120F9E7D41E002010B510461A46F7F72F
:1015400095FF002010BD00002DE9F0471B4F82469B
:101550000026387886B0002821D00024DFF860808B
:10156000A14600BF08EB0415A87B810702D410EA4E
:101570000A0F1BD00126284601F0BEF9B0B14FF684
:10158000FF71ADF802102988ADF80410862809D043
:1015900007218DF8001002906846FEF767FE06B03E
:1015A000BDE8F08706208DF80000F5E7641C022CEA
:1015B000D8D3002EF3D187F80090F0E7C41E0020A6
:1015C000482800202DE9F04707461E481C461546CE
:1015D00000780E4670B185B17CB1DFF86C804FF0B9
:1015E0000009A08802282BD200EB800118F8210006
:1015F00010BB19E00220BDE8F0870520FBE720685A
:101600001FB181883A8891420ED11EB1018832887B
:10161000914209D180682860206868600A482830B3
:10162000008928810020E6E7A088214600F05EF8C6
:101630000028E4D1C4F80090A088401CA080D0E726
:101640000A20D8E7881F0020682B0020F8B505463F
:101650004068244F0C46002648B32349CA6882429A
:1016600025D80969814222D3FBF7DAFEF8B128892F
:10167000398988421BD1D5E900018A68904216D188
:101680000020A7F1280200BF00EB800302EB8303D8
:101690005B688B4205D203F580538B4201D92080D1
:1016A00011E0401C80B20228EED30020F8BD268055
:1016B00000960AE0009829688068884205D1009861
:1016C0006860388928810120F8BD2088694600F0CB
:1016D0000DF80028EED12088401C80B2208002281E
:1016E000E6D3E2E7902B00203020002070B50E46B4
:1016F00000EB8001134800EB81004468306804F57A
:10170000805518B1418800EB810411E0083410E0E5
:1017100029462046FBF792FA20B1012805D002287D
:1017200007D10DE00120346070BD608804EB8004B7
:101730000C3429462046FBF794FA0028E8D170BD06
:10174000002070BD682B002038B50C4600210091A8
:1017500001460423074A0848FCF798FF08B10E2009
:1017600038BD064A04EB840102EB810101200874B4
:10177000002038BD102E020030200020682B0020F1
:1017800070B50C4B00210A4ADC680DE002EB8105C4
:101790008678AD78B54206D132F821500688B54238
:1017A00001D1586870BD491CA142EFD3002070BD23
:1017B00080230020941E00200A46FF2803D80146FB
:1017C0001046FFF76EBB70470846704770B501269C
:1017D00070044FF0E0210025C1F88001084C401052
:1017E000C4F84803C4F8080366602F20FDF7EAFE3A
:1017F000A660044C2F20A560FDF7E4FEA57070BD27
:1018000000100140401F00201FB501238DF800305B
:101810008DF808100192D0E90012684690471FBD6C
:1018200070B50D460446F8F75BF970B12846F8F735
:1018300069F968B16807000E002C0CDA04F00F019A
:1018400001F1E02181F8140D09E042F2010070BDC0
:1018500042F2020070BD04F1E02484F8000400208C
:1018600070BD000038B50021012548B101280CD019
:10187000032809D1FDF772FEBDE83840FCF758BCDB
:101880004FF0E020C0F8805138BD8DF80010684658
:10189000F8F7FAFB064C207808B9FCF72DFCE06855
:1018A000401CE060A5709DF80000F8F711FC38BD01
:1018B000F42800203EB5044609496846FDF7F4FDCA
:1018C00008E000BFD0E900212046904730B16846CB
:1018D000FDF701FE02980028F4D13EBD11203EBD67
:1018E000643002003EB5044608496846FDF7DCFD59
:1018F00007E000BFD0E90021204690476846FDF789
:10190000EAFD02980028F5D13EBD000070300200CB
:101910002DE9FC4104460C3000278046FBF770FBA4
:101920004FF6FF750646A842208803D1FBF758FB07
:10193000064602E03146FBF73DFB208800220121EC
:1019400000F0C6F8AE4212D06A4607213046FEF7D4
:1019500009FD60B9019D95F844003435C00705D1F3
:10196000414605F11200FBF710FB00B12F460023A2
:1019700020881A46394686DF05000BD000232088D0
:101980001A46314600F088F82088294600F01EF9F2
:10199000BDE8FC81002FFBD1002320881A46314688
:1019A00000F07AF82088002241F20601FAF788FB5D
:1019B000EEE700002DE9FC411D46089C16460F4647
:1019C000804644B16B46012207213846FEF7F4FCFD
:1019D000112801D010B10320BDE8FC8150210198ED
:1019E000F7F75DFD019806700198E56034302060DE
:1019F0000198183020610198401C60610748E0613F
:101A0000019940461131FBF759F90028E3D107212C
:101A10003846FEF75BFD0528DDD0DDE7B428002061
:101A2000002835D00278910701D411062FD4C2F3D3
:101A3000021104292BD8930703D5032901D11106DC
:101A400025D5437881788B4221D8072B1FD31029C5
:101A50001DD8C1784B071AD40079430717D40B0758
:101A600015D4030713D4D2074FEAC17201D042B193
:101A70000FE062B989070AD4C10708D1800706D4EC
:101A800007E0890705D4C10703D1800701D40020EE
:101A9000704701207047000070B50C4605466AB1DA
:101AA000002B12D009480122C1782846F8F772FFAE
:101AB00021462846BDE87040FBF77CBA002B04D0D5
:101AC000BDE870400846FBF777BA70BDD81E00200D
:101AD000F0B5174D14460F460A4685B006462978DC
:101AE000F8F758FF002F1FD00CB1012200E00022B0
:101AF00069783046F8F74EFF012C17D00022A978FC
:101B00003046F8F747FF0022E9783046F8F742FF01
:101B1000142208496846F7F7A9FCADF802608DF871
:101B200008406846FAF7CAFB05B0F0BD0122E6E7B7
:101B3000D81E0020A02D020038B50C4C2088A0F53E
:101B40007F41FF3911D06946FFF746F808B1F8F731
:101B500079F99DF80000800707D400212088FFF75D
:101B600077F8002801D0F8F76DF938BD481B002040
:101B700010B586B0044614216846F7F790FC04209F
:101B80008DF80000ADF802406846FAF797FB06B002
:101B900010BD000002498969002900D0084770473C
:101BA000EC22002030B585B00C46054614220649CB
:101BB0006846F7F75BFCADF8025068460294FAF706
:101BC00059FB05B030BD0000282D020030B585B0AE
:101BD0000C460546142206496846F7F747FCADF85F
:101BE000025068460294FAF769FB05B030BD000068
:101BF000B42D020010B5094C0020D2B2207004F1BF
:101C00000800FDF72FFE08B1F8F71CF960780028EE
:101C100002D021780029FAD010BD0000BC1F00209E
:101C20002DE9F0410746806A14468846C8B300256E
:101C300031E000BFB96A05EB450001EB8006B088D2
:101C4000801CFE2802D90C20BDE8F0812288401CAF
:101C500008F8020020881622401C80B2208008F874
:101C600000202088401C80B2208000EB08013088D2
:101C700000F098FC2188084480B22080B28842B1EC
:101C8000B16871B14044F7F7F1FB2088B18808448E
:101C900020806D1CEDB297F82C00A842CAD8002015
:101CA000D2E7FFE70720CFE710B50020F9F74AFB9E
:101CB00008B1F8F7C7F8F9F775FA08B1F8F7C2F8FC
:101CC00033DF002803D0BDE81040F8F7BBB810BDE3
:101CD00010B500F0B1F80548002203494078BDE88E
:101CE0001040F8F7F3BD0000C5D50100E01E00204C
:101CF00000F01CB910B51148FAF7DDFC0F48401C84
:101D0000FAF7D9FC0D48801CFAF7D5FC0B48C01C2B
:101D1000FAF7D1FC0948001DFAF7CDFC0748401D31
:101D2000FAF7C9FC0548401E8179182903D0012122
:101D3000C171002010BD032010BD0000E11E002075
:101D400000230A461946FBF79BBB000010B500783C
:101D5000114C0A2813D004DC082810D009281AD105
:101D60000DE00B280BD0132815D100220B49A079C8
:101D7000F8F7ACFD00220A49A078F8F7A7FD002289
:101D800006496079F8F7A2FD6078BDE810400022AE
:101D90000349F8F79BBD10BDE01E00203D02020084
:101DA000C5D5010070B50B4C05004FF001060CD0F5
:101DB000FFF736FE58B1286820612879207504F1B4
:101DC0001000A0602670002070BD0020F9E70720F9
:101DD00070BD0000E01E002010B504460078052804
:101DE00002D0122821D105E06088A168BDE810402A
:101DF00000F060B90F480021806880B10D48237A57
:101E00001030007800F0010203B101239A4206D39A
:101E1000627AC0F3400002B10122904200D2012157
:101E2000608801230022FBF72BFB2046BDE8104011
:101E3000FAF752BAE01E002030B50446008885B09B
:101E400014284FD00ADC11282CD0132828D134F8BC
:101E5000040FF8F761FD01282FD038E0192847D08A
:101E60001A281DD1A088FEF7E3F9002818D1A08810
:101E7000F8F71CFD0028A0884BD02A4900220978D9
:101E8000F8F788FD02208DF80000A088ADF8020068
:101E900000208DF808008DF809006846FAF70EFA60
:101EA00005B030BD207A3D2804D04FF48851A08879
:101EB000002224E041F23D01F9E72079C00701D07A
:101EC000012200E0022220880121FFF701FE34F800
:101ED000045B142214496846F7F7C8FAADF80250BB
:101EE0000294DAE705B0201DBDE83040FFF710BDD1
:101EF000217A201D41B14279008802F0030205B029
:101F0000BDE83040FBF718BB05B0BDE83040F8F73E
:101F10003FB905B00122BDE8304041F20601FAF7B1
:101F2000CFB80000D81E0020DC2D02000A7802493C
:101F30000979F8F72FBD0000D81E002010B514480D
:101F4000FAF7B0FB1248401CFAF7ACFB1048801CB3
:101F5000FAF7A8FB0E48C01CFAF7A4FB0C48001DBA
:101F6000FAF7A0FB0A48017818290FD04178182900
:101F70000CD08178182909D0C178182906D00179A8
:101F8000182903D001214171002010BD032010BD8C
:101F9000D81E002070B50C460546F8F7BDFC012898
:101FA00002D043F2020070BD21004FF00000FAD0D1
:101FB00028467EDF70BD00002DE9F74F8AB09246BB
:101FC00088460A98F8F7A8FC06464FF6FF790024E1
:101FD0004D4627460A98FEF7D3FB8346202101A8E9
:101FE000F7F75DFA012E01D0DEB105E02F4800229F
:101FF00001790A98F8F7CEFCB8F1000F16D098F8DE
:102000000000C00714D00A98FAF7EAFF05464845D1
:1020100016D1FEF79DF9054648450ED04FF0010B4D
:102020000CE043F202000DB0BDE8F08F852721E0FF
:102030001F48CDF810A008901CE003246CB121E0EB
:10204000012E0AD10A98F7F76BFE30B90A98FFF70C
:102050008FFD0A98F7F764FE50B101A8009053462F
:10206000324629460A98FFF7A5FC040002D009E091
:10207000852712E0012E10D001AB002239460A98C4
:102080007FDF044654EA07000DD000225B46294654
:102090000A98FFF701FD2046C5E701AB42463946E5
:1020A0000A987FDFEDE70122F0E70000D81E00204C
:1020B000B42800203EB505460C466846FBF7B6FD41
:1020C0006A4621462846FEF7BCF809480099C268CE
:1020D0002846FFF771FF0446014601222846FAF719
:1020E00007FB21462846009AFAF78AF83EBD000011
:1020F000E01E0020002805D103490120487000207F
:10210000F9F734BB70470000F428002010B5162002
:10211000F7F7E6FC48B10A4882684FF4800152B1F3
:10212000016821F48001016010BDBDE8104042F259
:102130000100F7F787BE4FF0E020C0F8801110BD16
:10214000B42A002010B51620F7F7CAFC80B10F485A
:1021500090F800044009F7F7D5FC60B10C4882689C
:102160004FF480016AB1016841F48001016010BD43
:1021700042F2010001E042F20200BDE81040F7F730
:1021800061BE4FF0E020C0F8001110BD16E000E085
:10219000B42A00202DE9F84F204D92468946064684
:1021A0009846012269461846AF68F9F701FA58B314
:1021B000009800210446801C09E000BF00EA0703E4
:1021C0005AF8212005EB8303401C491CDA60414585
:1021D000F4D34FEA164AF9F749FF4AEA0041601C76
:1021E000384005EB80003C4005EB8402C160D068BC
:1021F00066F3C50068F3891069F39F2020F003009F
:10220000401C20F00400D06095F8200402E000BFDC
:10221000FCF788FC0028FBD1BDE8F88F4C2D00208E
:1022200010B50446082902D00020F7F70BFED4E9C8
:102230000010BDE8104008472DE9F84F1D4C00255F
:102240006846D4E901A6F9F71BFF002738B300233D
:10225000009A61681CE0D1F800C00846944503D993
:10226000ACEB02020A6015E0A2EB0C0263440760CB
:10227000D0F80CC0C1698146BCF1000F08D006EB54
:10228000030828F07F48C0E9018CC9F81C500546B6
:102290000029E0D128466160FBF7AAF903E028464F
:1022A000FBF7A6F910B15046F9F782FAE770BDE8DE
:1022B000F88F0000401F00200D4B10B5596831B158
:1022C00002680C68A24204D8A21A0A60C161586070
:1022D00010BD0B4603E00B46C969121B21B10C6807
:1022E0009442F8D3A41A0C600260C161D86110BD99
:1022F000401F00202DE9F041144E77683D462C46E2
:1023000003E0844204D02546E469002CF9D11BE0A7
:10231000D4B1A5420BD1F869706040B90C490120D5
:1023200088600021B160F0702F20FDF74BF9216823
:10233000E069E86110B10268114401607068874289
:1023400002D00120BDE8F0810020FBE7401F002003
:10235000001001407CB5064600240D468DF8004073
:102360006846F7F791FE01A800F0EEF970B105702C
:10237000094946609DF8040048709DF80000F7F791
:10238000A7FE1420F7F7C0F920467CBD04249DF871
:102390000000F7F79DFEF7E7A82900202DE9FC4192
:1023A0001D4D6C68002C35D01C4800270068A968BA
:1023B000B846401A20F07F462068B04215D8361A39
:1023C00007442046E469017C69B180F810804169C6
:1023D000009180690190124A08216846F7F73EFD96
:1023E00008B1F7F72FFD002CE6D1297868788142F3
:1023F00006D1401CC0B26870022801D185F8018066
:10240000054869780C3040F82170BDE8FC41142083
:10241000F7F77AB9BDE8FC81401F002004150140A0
:10242000212202000149012008707047BC1F0020D2
:1024300010B588B0044620220E496846F7F716F812
:1024400006200090C01F0190029003904FF0EB70A7
:1024500006900CB1084A00E0002269460748FBF7E5
:102460007FFE08B1F7F7EEFC0448001F447008B087
:1024700010BD00003030020025240200C01F0020E3
:102480001FB50A4601788DF8001041680191017A64
:102490008DF80810C0680390044850F82210001FFF
:1024A00050F82220684690471FBD0000001F002002
:1024B0002DE9FF410C464FF4927705463946FDF76A
:1024C00041F80026C0B139462846FDF740F8022001
:1024D0008DF80000D5F88004C5F880040390D5F885
:1024E0003C058DF80800E0680190A661E661D4E93A
:1024F00000126846904723E04FF488773946284613
:10250000FDF720F8E0B139462846FDF720F8D5F868
:102510003C15A069884213D1E06960B1E268D5F842
:10252000000220F02000C5F80002E069A0612069E7
:10253000E661E06001E0A661E2682046FFF764F929
:102540004FF4A27739462846FCF7FCFF60B13946C4
:102550002846FCF7FCFFA06930B1A661D5F83C1510
:102560002046E268FFF750F94FF490773946284645
:10257000FCF7E8FF002813D039462846FCF7E7FFB0
:10258000606900280CD0D5F84C058DF800608DF8F6
:102590000800A06801906661D4E90012684690477F
:1025A000BDE8FF810870000A4870022070470000F3
:1025B00010B514210448F6F772FF04480068FBF7D1
:1025C00057FB002010BD00002C2C0020942E020090
:1025D0002DE9F05F8346DDE90A4A994690460D46AB
:1025E0000846012703E000BFB0FBF8F07F1C404520
:1025F000FAD2B94500D94F465FEACA7012D18CB100
:102600005FEA8A7002D5B9F1000F01D0202607E0F9
:10261000302605E031465846641EF9F711F80CB132
:10262000A742F7D35FF00106B9F1010F02D9A9F172
:10263000010903E0B5FBF6F0404502D306FB08F6BE
:10264000F2E7DFF83C9000BFB5FBF6F000FB165553
:1026500019F800105846F8F7F3FFB6FBF8F6002E0D
:10266000F2D15FEACA7009D0002C07D0A74205D288
:1026700020215846641EF8F7E3FFF5E7BDE8F09F18
:10268000242E02000348002201498078F8F71EB981
:1026900021BD0100A41E0020F8B5054680B2FAF75E
:1026A000A1FD040013D0154E207A0027317B88420B
:1026B0000ED2A8B204F10A0175DF28B1112806D0A4
:1026C000BDE8F840FFF766BA207A401C2072F8BDDA
:1026D0002772307C38B1A8B23B2176DF18B10828C8
:1026E00001D0FFF757FA71690029F0D08DF800701A
:1026F000ADF8025068468847F8BD0000EC22002083
:10270000417939B190F8B21021B990F8B40008B10C
:10271000012070470020704701460148FBF72FBB9E
:102720000823002030B40446007A00280AD06088CC
:10273000002166DF28B1112802D0616830BC08474B
:102740000120207230BC70470A494A788B78521CAD
:10275000D2B2934200D100220B78934201D10020E3
:1027600070470270487800EB400001EBC000001D8C
:1027700070470000A82900202DE9FC411646DDE93C
:102780000854CDE900541F468046022200F00CF8A0
:10279000002807D1CDE900543B461022314640467F
:1027A00000F002F8BDE8FC812DE9FC5F0026DDE9C0
:1027B0000C4B994692468E4680462788354630E037
:1027C000D8F80400002200EB8500694600680190FB
:1027D00001A864DF002830D19DF8000050451FD1CA
:1027E0000EB1002100E00221228808441118594549
:1027F00022D846B9521C90B2208009F800E0208807
:10280000401C20800126218801A801EB09026946AD
:1028100064DF002811D120889DF800100844208032
:102820006D1CB8F80000A842CADC56B12088C01B55
:10283000401E80B2FF2802D90C20BDE8FC9F09F899
:1028400007000020F9E710B5042817D209B10324C6
:1028500000E00024F8F7F4FB4FF0A04101EB80000A
:10286000D0F8001721F44031C0F80017D0F8001755
:1028700041EA0441C0F80017002010BD062010BD39
:10288000002070472DE9F84F114D884681461E46BD
:1028900017466946DDF828A02868FBF704FA04000B
:1028A00013D01C21F6F7FBFD00202071C4F8009026
:1028B000C4E90486C4E902A769462868FBF714FA4C
:1028C000FEF714FE0020BDE8F88F0420FBE70000AF
:1028D000942E020082780121012A0BD0062A09D009
:1028E000072A06D0082A06D1416889880931890853
:1028F00000E01421018070471CB5044600200090C0
:102900000190A0788DF80200617B1A48FEF734F937
:10291000020017D0237BA1786846FDF737FF684691
:10292000FFF7D8FF208804F1080369466268FDF7C5
:10293000ABFE48B1072806D001210F4A112808D064
:1029400086280FD003201CBDA17B21F00301A173B9
:102950001CBDA07B20F0010040F00200A0731170AC
:1029600000201CBDA37B23F0020343F00103A373EB
:1029700011701CBD38280020C41E002038B5054643
:102980000C46002001E00098401C00906946284653
:1029900000F00EF800280AD08178A142F3D1817BA3
:1029A0008A07F0D4C907EED181680029EBD138BD80
:1029B00010B5084B0A6809E003EB0214248884422E
:1029C00003D103EB02100A6010BD521C022AF3D39C
:1029D000002010BD482800204FF6FF710180FF2124
:1029E00081704173817B21F00301817300210173A8
:1029F000416081607047000070B50546002406E024
:102A0000687B2044C1B20648FEF7CAF8641C287BE4
:102A1000A042F5D82846BDE87040FFF7DDBF0000B2
:102A2000382800202DE9FC470646364898461446CB
:102A300000780D464FF0000978B37DB32888A0F5E3
:102A40007F41FF3931D0688848B36868FAF7E8FCFD
:102A500068B374B32088ADF80000678801A8FEF75A
:102A600077FC04002FD084F800804FF0000A84F82F
:102A700016A0BDF80000A0826868206121480121ED
:102A80000C38FBF79AF9E060288820816888A080DC
:102A9000E780B8F1030F1DD020E001E003E004E07F
:102AA0000220BDE8FC870520FBE70420F9E70320AE
:102AB000F7E7FFE72889694687B2384600F0ACF8A7
:102AC0000028EED1CAE7BDF80010384600F098F8AB
:102AD0000820E6E70420A0753068A061A4F80A90F9
:102AE00001A8FEF743FC46B1C6F804A0E168064819
:102AF000316086F80AA000893081FEF7E9FC0020E9
:102B0000CFE70000881F0020902B00202DE9F8431C
:102B10000D46898A374A01EB810102EB810630B10B
:102B200029463046FDF792FA0120BDE8F883318945
:102B30007068002400EB81072E48A97DA8384FF06B
:102B40000E0807294ED2DFE801F00D2D16240440AF
:102B50004A004460A969016026482749A838FEF761
:102B600075FD30B10220A875042339462A1D009452
:102B700023E00A20D9E728692A4608B1032000E0AB
:102B800001209075042305F10C0207F1080100945F
:102B900013E00120A8750094E88807F10C01830078
:102BA0002A690AE028782A4603280CD00620907566
:102BB000042305F10802391D00941048FBF766FD57
:102BC000A8B144460FE00520F1E70621A9750A499E
:102BD00040680988FEF7B8FD040004D107E041F61B
:102BE0001D5400E00F2429463046FDF72FFA2046F9
:102BF0009BE70000682B0020681F00203020002089
:102C000001EB8102034901EB82014A89101AC01EBF
:102C100048817047682B002070B5C01C82B240F21A
:102C2000FE30824201D3092070BD114B00204FF4C9
:102C3000806500BF00EB800413F8246096B903EBB5
:102C400084063489768914443444A4B2AC4209D24F
:102C5000088000EB800003EB800041891144418132
:102C6000002070BD401C80B20228E3D3072070BD55
:102C7000682B002088200020111213140D0E0F1055
:102C80004C2200206C220020982200200D0003001E
:102C9000C5B101000E000300C5B101000F00030023
:102CA000C5B1010010000300C5B101000100000022
:102CB0000000000000000000000000000000000014
:102CC0000000000000000000000000000000000004
:102CD00000000000000000000000000000000000F4
:102CE00000000000000000000000000000000000E4
:102CF00000000000000000000000000000000000D4
:102D000000000000000000000000000000000000C3
:102D100000000000000000000000000000000000B3
:102D2000000000000000000007000000000000009C
:102D3000000000000000000000000000060000008D
:102D40000000000000000000000000000000000083
:102D5000DD0D0200ADC90100770A0000000000008F
:102D6000770A000000000000DD02020007000000FA
:102D70000000000000000000000000000000000053
:102D8000F10E02004D1D02000DCA010001000000FD
:102D90000000000001000600D41E0020D91D020022
:102DA0000100000000000000000000000000000022
:102DB000000000000700000000000000000000000C
:102DC0000000000000000000030000000000000000
:102DD00000000000000000000000000005000000EE
:102DE00000000000000000000000000000000000E3
:102DF0003112020000000050B19A010003000000EF
:102E0000882900200738FDD870470000541F002093
:102E10000000FFFFDEC0ADDEFF011EF1DEC0ADDE53
:102E2000FE011EF130313233343536373839414204
:102E3000434445466E72665F6673746F7261676580
:102E40005F696E6974006E72665F6673746F72613B
:102E500067655F756E696E6974006E72665F667332
:102E6000746F726167655F72656164006E72665F40
:102E70006673746F726167655F7772697465006EFF
:102E800072665F6673746F726167655F65726173A6
:102E900065000000981F00200010000004000000E2
:102EA00001000000E9D00100B1250200391502003F
:102EB00085280200CDC00100C91702008128020048
:102EC0006DD30100000000000000000000000000C1
:102ED000000000000000000000000000C42E0200FE
:102EE000DC2E020004000000556E6B6E6F776E20C2
:102EF0006572726F7220636F6465000000000000ED
:102F0000FC35020001000000A834020002000000AD
:102F10009C320200030000001C3502000400000087
:102F20007035020005000000503402000600000069
:102F3000EC330200070000005835020008000000D2
:102F40006434020009000000C83402000A000000D6
:102F5000E43502000B000000843202000C00000087
:102F60007C3402000D0000004C3602000E00000010
:102F7000483502000F0000008435020010000000F8
:102F8000B835020011000000603602001200000097
:102F90003436020013000000D0350200800000002B
:102FA000043402008100000040330200820000006F
:102FB0000033020083000000E032020084000000C1
:102FC0001C33020085000000283402008600000047
:102FD0003035020090000000CC3302009100000068
:102FE000C032020092000000903402000082000013
:102FF0009835020001820000E434020002820000E1
:1030000000350200008400005C33020001840000EF
:103010000836020002840000A4330200038400008A
:1030200080330200C1EA0100A9EA0100A1EA01001F
:10303000FFFFFFFFFFFFFFFFFFFFFFFFFFFFFFFFA0
:1030400000000000000000000000D60107000000A2
:10305000303A0200383A0200000000000000000090
:10306000010000075030020060300200080000003C
:1030700088300200983002000800000098300200FA
:10308000A830020008000000603A0200703A020016
:103090000000000000000000503A0200603A020008
:1030A0000000000000000000E0390200E8390200E2
:1030B000E8390200183A0200183A0200283A0200E1
:1030C000283A0200303A0200481B0020A8300200D3
:1030D000C830020008000000383A0200483A0200F6
:1030E000483A0200503A0200D8300200E8300200AC
:1030F0000800000000404040404040404040414106
:1031000041414140404040404040404040404040BC
:103110004040404040050202020202020202020256
:103120000202020202202020202020202020200253
:1031300002020202020290909090909010101010E3
:10314000101010101010101010101010101010107F
:103150000202020202028888888888880808080813
:1031600008080808080808080808080808080808DF
:103170000202020240000000F53002004A756E654E
:10318000000000004D6172636800000041707269C8
:103190006C000000556E6B6E6F776E004465636562
:1031A0006D6265720000000053657074656D626544
:1031B000720000004E6F76656D626572000000005F
:1031C0004F63746F626572004175677573740000B8
:1031D0004D61790046726964617900004D6F6E64DB
:1031E0006179000053756E646179000053617475F4
:1031F00072646179000000005765646E65736461F4
:1032000079000000547565736461790054687572C3
:1032100073646179000000004A756C790000000059
:103220004A616E7561727900466562727561727984
:1032300000000000616464725F69735F776974689D
:10324000696E5F626F756E647328705F66732C20A1
:10325000706167655F616464722C20286C656E2004
:103260002A20705F66732D3E705F666C6173685FC5
:10327000696E666F2D3E65726173655F756E697408
:10328000292900004E52465F4552524F525F494E27
:1032900056414C49445F4441544100004E52465F00
:1032A0004552524F525F534F465444455649434549
:1032B0005F4E4F545F454E41424C45440000000074
:1032C0004E52465F4552524F525F46454154555209
:1032D000455F4E4F545F454E41424C45440000000F
:1032E0004E52465F4552524F525F4D555445585FBE
:1032F000554E4C4F434B5F4641494C4544000000FE
:103300004E52465F4552524F525F4D555445585F9D
:103310004C4F434B5F4641494C4544004E52465F3B
:103320004552524F525F4D555445585F434F4E449E
:103330005F494E49545F4641494C454400000000F6
:103340004E52465F4552524F525F4D555445585F5D
:10335000494E49545F4641494C4544004E52465FF0
:103360004552524F525F424C455F495053505F5255
:10337000585F504B545F5452554E4341544544009E
:103380004E52465F4552524F525F424C455F495044
:1033900053505F504545525F52454A45435445445A
:1033A000000000004E52465F4552524F525F424C61
:1033B000455F495053505F4C494E4B5F444953431E
:1033C0004F4E4E4543544544000000004E52465F68
:1033D0004552524F525F4150495F4E4F545F494DE5
:1033E000504C454D454E5445440000004E52465FFA
:1033F0004552524F525F4E4F545F535550504F52AB
:10340000544544004E52465F4552524F525F4D4F15
:1034100044554C455F4E4F545F494E495449414CC9
:10342000495A4544000000004E52465F4552524FF3
:10343000525F4D4F44554C455F414C5245414459B4
:103440005F494E495449414C495A454400000000E7
:103450004E52465F4552524F525F4E4F545F464F59
:10346000554E44004E52465F4552524F525F494EB0
:1034700056414C49445F5354415445004E52465FB7
:103480004552524F525F444154415F53495A45009F
:103490004E52465F4552524F525F494F5F50454E24
:1034A00044494E47000000004E52465F4552524F7D
:1034B000525F5356435F48414E444C45525F4D491D
:1034C0005353494E470000004E52465F4552524FFB
:1034D000525F494E56414C49445F4C454E47544813
:1034E000000000004E52465F4552524F525F445218
:1034F000565F5457495F4552525F414E41434B001E
:103500004E52465F4552524F525F4452565F545797
:10351000495F4552525F444E41434B004E52465F15
:103520004552524F525F494E5445524E414C000055
:103530004E52465F4552524F525F53544F5241478D
:10354000455F46554C4C00004E52465F4552524F27
:10355000525F4E554C4C00004E52465F4552524F02
:10356000525F494E56414C49445F504152414D00D3
:103570004E52465F4552524F525F4E4F5F4D454D42
:10358000000000004E52465F4552524F525F464F78
:103590005242494444454E004E52465F4552524FB6
:1035A000525F4452565F5457495F4552525F4F56DF
:1035B000455252554E0000004E52465F4552524F02
:1035C000525F494E56414C49445F414444520000C9
:1035D0004E52465F4552524F525F5245534F5552DD
:1035E000434553004E52465F4552524F525F494E3B
:1035F00056414C49445F464C414753004E52465F4A
:1036000053554343455353004E52465F4552524F24
:10361000525F424C455F495053505F4348414E4EC4
:10362000454C5F414C52454144595F4558495354BC
:10363000530000004E52465F4552524F525F434F77
:103640004E4E5F434F554E54000000004E52465FB1
:103650004552524F525F54494D454F55540000005A
:103660004E52465F4552524F525F425553590000E9
:103670007761726E696E670064656275670000004D
:103680001B5B313B33306D001B5B306D0000000075
:103690001B5B313B33316D001B5B313B33326D00C3
:1036A0001B5B313B33336D001B5B313B33346D00AF
:1036B0001B5B313B33356D001B5B313B33366D009B
:1036C0001B5B313B33376D00696E666F0000000095
:1036D0006572726F7200000073645F626C655F6395
:1036E00066675F73657428292072657475726E65EC
:1036F00064202573207768656E20617474656D7031
:1037000074696E6720746F2073657420424C455F46
:1037100047415454535F4346475F534552564943CC
:10372000455F4348414E4745442E000073645F6245
:103730006C655F6366675F736574282920726574C2
:1037400075726E6564202573207768656E206174DC
:1037500074656D7074696E6720746F207365742072
:10376000424C455F434F4D4D4F4E5F4346475F567A
:10377000535F555549442E0073645F626C655F6307
:1037800066675F73657428292072657475726E654B
:1037900064202573207768656E20617474656D7090
:1037A00074696E6720746F2073657420424C455FA6
:1037B00047415454535F4346475F415454525F540A
:1037C00041425F53495A452E0000000073645F6216
:1037D0006C655F6366675F73657428292072657422
:1037E00075726E6564202573207768656E2061743C
:1037F00074656D7074696E6720746F2073657420D2
:10380000424C455F434F4E4E5F4346475F474150F2
:103810002E00000073645F626C655F6366675F73B0
:10382000657428292072657475726E65642025732D
:10383000207768656E20617474656D7074696E6759
:1038400020746F2073657420424C455F4741505F80
:103850004346475F524F4C455F434F554E542E00F1
:10386000626C655F64625F64697363006E72665F59
:10387000626C655F6761747400000000626C655F74
:103880006374735F63000000636C6F636B00000020
:10389000434C4F434B0000004750494F54450000F4
:1038A00050525300554152544500000061746669FE
:1038B000666F2E6D5F717565756500006E72665F6F
:1038C0006673746F726167650000000061746669F9
:1038D000666F2E6D5F6669666F0000007077725FBD
:1038E0006D676D740000000062616C6C6F632E6C1C
:1038F0006F675F6D656D706F6F6C00006170700059
:103900006E72665F736468006E72665F7364685F90
:10391000626C65006E72665F7364685F736F6300EC
:10392000703A0200481B002040050000209501006D
:10393000143B020088200020E8180000D09A010003
:1039400060380200000003036C380200000003032B
:103950007C380200000003038838020000000000E9
:1039600090380200000000009838020000000000BB
:10397000A038020000000000A4380200000000008F
:10398000AC38020000000003BC3802000000030352
:10399000CC38020000000003DC3802000000000008
:1039A000E838020000000003FC38020000000303B6
:1039B000003902000000030308390200000003037D
:1039C0001439020000000303E01F0020D81F00206C
:1039D000E01F00208C2C0020742000201800000024
:1039E0000DAF010000000000FDDE01006821002095
:1039F0003BA5010084210020B5AB0100541B002031
:103A0000A1AD01000000000011AE010000000000A7
:103A100011B00100000000005FAA01005821002041
:103A200023E0010078210020CDAC0100000000005F
:103A3000B1E5010000000000F520020000000000D8
:103A4000E9E5010000000000A5A501008421002097
:103A5000E1F20100000000006DF401000000000030
:103A60006518020000000000C9E501000000000028
:103A700023FFFF04FF05180101FF01D116FFFF948A
:103A800031021ADC04140432021AF8081A0C081A5B
:103A9000D4081AEC041AE40429201A20141A280461
:103AA0001A840C1A8C041AD0041A7C041A18141ADA
:103AB000C8081AA8041AC0041AB4041A9C040138CD
:103AC0000B28D90D3C2A18017909390A01791364A8
:103AD000200240200A1A6C4412204240042524305F
:103AE0000214D036021A70041AC8041A78041A880C
:103AF000041A80041A90041A98041AA0041AA8043C
:103B00001AB0041AB8041AC004518490D003044DAA
:043B100075C7010074
:040000050001920163
:00000001FF
